 AsyncInvokers

 Timestamp is 01b2b90b (reproducible build file hash)

 Preferred load address is 0000000180000000

 Start         Length     Name                   Class
 0001:00000000 00001710H .text$mn                CODE
 0001:00001710 00000036H .text$mn$00             CODE
 0001:00001746 00000092H .text$x                 CODE
 0002:00000000 00000128H .idata$5                DATA
 0002:00000128 00000038H .00cfg                  DATA
 0002:00000160 00000008H .CRT$XCA                DATA
 0002:00000168 00000008H .CRT$XCZ                DATA
 0002:00000170 00000008H .CRT$XIA                DATA
 0002:00000178 00000008H .CRT$XIZ                DATA
 0002:00000180 00000008H .CRT$XPA                DATA
 0002:00000188 00000008H .CRT$XPZ                DATA
 0002:00000190 00000008H .CRT$XTA                DATA
 0002:00000198 00000008H .CRT$XTZ                DATA
 0002:000001a0 00000000H .gehcont$y              DATA
 0002:000001a0 00000000H .gfids$y                DATA
 0002:000001a0 00000260H .rdata                  DATA
 0002:00000400 00000000H .rdata$CastGuardVftablesA DATA
 0002:00000400 00000000H .rdata$CastGuardVftablesC DATA
 0002:00000400 000000acH .rdata$voltmd           DATA
 0002:000004ac 0000029cH .rdata$zzzdbg           DATA
 0002:00000748 00000008H .rtc$IAA                DATA
 0002:00000750 00000008H .rtc$IZZ                DATA
 0002:00000758 00000008H .rtc$TAA                DATA
 0002:00000760 00000008H .rtc$TZZ                DATA
 0002:00000768 00000268H .xdata                  DATA
 0002:000009d0 00000974H .edata                  DATA
 0002:00001344 00000050H .idata$2                DATA
 0002:00001394 00000014H .idata$3                DATA
 0002:000013a8 00000128H .idata$4                DATA
 0002:000014d0 00000312H .idata$6                DATA
 0003:00000000 00000040H .data                   DATA
 0003:00000040 000005f8H .bss                    DATA
 0004:00000000 0000039cH .pdata                  DATA

  Address         Publics by Value              Rva+Base               Lib:Object

 0000:00000000       __AbsoluteZero             0000000000000000     <absolute>
 0000:00000000       ___safe_se_handler_count   0000000000000000     <absolute>
 0000:00000000       ___safe_se_handler_table   0000000000000000     <absolute>
 0000:00000000       __arm64x_extra_rfe_table   0000000000000000     <absolute>
 0000:00000000       __arm64x_extra_rfe_table_size 0000000000000000     <absolute>
 0000:00000000       __arm64x_native_entrypoint 0000000000000000     <absolute>
 0000:00000000       __arm64x_redirection_metadata 0000000000000000     <absolute>
 0000:00000000       __arm64x_redirection_metadata_count 0000000000000000     <absolute>
 0000:00000000       __dynamic_value_reloc_table 0000000000000000     <absolute>
 0000:00000000       __enclave_config           0000000000000000     <absolute>
 0000:00000000       __guard_check_icall_a64n_fptr 0000000000000000     <absolute>
 0000:00000000       __guard_eh_cont_count      0000000000000000     <absolute>
 0000:00000000       __guard_eh_cont_table      0000000000000000     <absolute>
 0000:00000000       __guard_fids_count         0000000000000000     <absolute>
 0000:00000000       __guard_fids_table         0000000000000000     <absolute>
 0000:00000000       __guard_iat_count          0000000000000000     <absolute>
 0000:00000000       __guard_iat_table          0000000000000000     <absolute>
 0000:00000000       __guard_longjmp_count      0000000000000000     <absolute>
 0000:00000000       __guard_longjmp_table      0000000000000000     <absolute>
 0000:00000000       __hybrid_auxiliary_iat     0000000000000000     <absolute>
 0000:00000000       __hybrid_auxiliary_iat_copy 0000000000000000     <absolute>
 0000:00000000       __hybrid_code_map          0000000000000000     <absolute>
 0000:00000000       __hybrid_code_map_count    0000000000000000     <absolute>
 0000:00000000       __x64_code_ranges_to_entry_points 0000000000000000     <absolute>
 0000:00000000       __x64_code_ranges_to_entry_points_count 0000000000000000     <absolute>
 0000:00000100       __guard_flags              0000000000000100     <absolute>
 0000:00000000       __ImageBase                0000000180000000     <linker-defined>
 0001:00000000       ??$launch@HP6AHXZ@@YAHP6AHXZ@Z 0000000180001000 f i libAsyncInvokers.obj
 0001:00000030       ??$launch@MP6AMXZ@@YAMP6AMXZ@Z 0000000180001030 f i libAsyncInvokers.obj
 0001:00000060       ??$launch@NP6ANXZ@@YANP6ANXZ@Z 0000000180001060 f i libAsyncInvokers.obj
 0001:00000090       ??$launch@PEAXP6APEAXXZ@@YAPEAXP6APEAXXZ@Z 0000000180001090 f i libAsyncInvokers.obj
 0001:000000c0       ??$launch@US_D@@P6A?AU1@XZ@@YA?AUS_D@@P6A?AU0@XZ@Z 00000001800010c0 f i libAsyncInvokers.obj
 0001:000000c0       ??$launch@US_FF@@P6A?AU1@XZ@@YA?AUS_FF@@P6A?AU0@XZ@Z 00000001800010c0 f i libAsyncInvokers.obj
 0001:000000c0       ??$launch@US_FI@@P6A?AU1@XZ@@YA?AUS_FI@@P6A?AU0@XZ@Z 00000001800010c0 f i libAsyncInvokers.obj
 0001:000000c0       ??$launch@US_IF@@P6A?AU1@XZ@@YA?AUS_IF@@P6A?AU0@XZ@Z 00000001800010c0 f i libAsyncInvokers.obj
 0001:000000c0       ??$launch@US_II@@P6A?AU1@XZ@@YA?AUS_II@@P6A?AU0@XZ@Z 00000001800010c0 f i libAsyncInvokers.obj
 0001:000000c0       ??$launch@US_P@@P6A?AU1@XZ@@YA?AUS_P@@P6A?AU0@XZ@Z 00000001800010c0 f i libAsyncInvokers.obj
 0001:000000f0       ??$launch@US_DD@@P6A?AU1@XZ@@YA?AUS_DD@@P6A?AU0@XZ@Z 00000001800010f0 f i libAsyncInvokers.obj
 0001:000000f0       ??$launch@US_DF@@P6A?AU1@XZ@@YA?AUS_DF@@P6A?AU0@XZ@Z 00000001800010f0 f i libAsyncInvokers.obj
 0001:000000f0       ??$launch@US_DFF@@P6A?AU1@XZ@@YA?AUS_DFF@@P6A?AU0@XZ@Z 00000001800010f0 f i libAsyncInvokers.obj
 0001:000000f0       ??$launch@US_DFI@@P6A?AU1@XZ@@YA?AUS_DFI@@P6A?AU0@XZ@Z 00000001800010f0 f i libAsyncInvokers.obj
 0001:000000f0       ??$launch@US_DI@@P6A?AU1@XZ@@YA?AUS_DI@@P6A?AU0@XZ@Z 00000001800010f0 f i libAsyncInvokers.obj
 0001:000000f0       ??$launch@US_DIF@@P6A?AU1@XZ@@YA?AUS_DIF@@P6A?AU0@XZ@Z 00000001800010f0 f i libAsyncInvokers.obj
 0001:000000f0       ??$launch@US_DII@@P6A?AU1@XZ@@YA?AUS_DII@@P6A?AU0@XZ@Z 00000001800010f0 f i libAsyncInvokers.obj
 0001:000000f0       ??$launch@US_FD@@P6A?AU1@XZ@@YA?AUS_FD@@P6A?AU0@XZ@Z 00000001800010f0 f i libAsyncInvokers.obj
 0001:000000f0       ??$launch@US_FFD@@P6A?AU1@XZ@@YA?AUS_FFD@@P6A?AU0@XZ@Z 00000001800010f0 f i libAsyncInvokers.obj
 0001:000000f0       ??$launch@US_FID@@P6A?AU1@XZ@@YA?AUS_FID@@P6A?AU0@XZ@Z 00000001800010f0 f i libAsyncInvokers.obj
 0001:000000f0       ??$launch@US_ID@@P6A?AU1@XZ@@YA?AUS_ID@@P6A?AU0@XZ@Z 00000001800010f0 f i libAsyncInvokers.obj
 0001:000000f0       ??$launch@US_IFD@@P6A?AU1@XZ@@YA?AUS_IFD@@P6A?AU0@XZ@Z 00000001800010f0 f i libAsyncInvokers.obj
 0001:000000f0       ??$launch@US_IID@@P6A?AU1@XZ@@YA?AUS_IID@@P6A?AU0@XZ@Z 00000001800010f0 f i libAsyncInvokers.obj
 0001:00000150       ??$launch@US_DDD@@P6A?AU1@XZ@@YA?AUS_DDD@@P6A?AU0@XZ@Z 0000000180001150 f i libAsyncInvokers.obj
 0001:00000150       ??$launch@US_DDF@@P6A?AU1@XZ@@YA?AUS_DDF@@P6A?AU0@XZ@Z 0000000180001150 f i libAsyncInvokers.obj
 0001:00000150       ??$launch@US_DDI@@P6A?AU1@XZ@@YA?AUS_DDI@@P6A?AU0@XZ@Z 0000000180001150 f i libAsyncInvokers.obj
 0001:00000150       ??$launch@US_DFD@@P6A?AU1@XZ@@YA?AUS_DFD@@P6A?AU0@XZ@Z 0000000180001150 f i libAsyncInvokers.obj
 0001:00000150       ??$launch@US_DID@@P6A?AU1@XZ@@YA?AUS_DID@@P6A?AU0@XZ@Z 0000000180001150 f i libAsyncInvokers.obj
 0001:00000150       ??$launch@US_FDD@@P6A?AU1@XZ@@YA?AUS_FDD@@P6A?AU0@XZ@Z 0000000180001150 f i libAsyncInvokers.obj
 0001:00000150       ??$launch@US_FDF@@P6A?AU1@XZ@@YA?AUS_FDF@@P6A?AU0@XZ@Z 0000000180001150 f i libAsyncInvokers.obj
 0001:00000150       ??$launch@US_FDI@@P6A?AU1@XZ@@YA?AUS_FDI@@P6A?AU0@XZ@Z 0000000180001150 f i libAsyncInvokers.obj
 0001:00000150       ??$launch@US_IDD@@P6A?AU1@XZ@@YA?AUS_IDD@@P6A?AU0@XZ@Z 0000000180001150 f i libAsyncInvokers.obj
 0001:00000150       ??$launch@US_IDF@@P6A?AU1@XZ@@YA?AUS_IDF@@P6A?AU0@XZ@Z 0000000180001150 f i libAsyncInvokers.obj
 0001:00000150       ??$launch@US_IDI@@P6A?AU1@XZ@@YA?AUS_IDI@@P6A?AU0@XZ@Z 0000000180001150 f i libAsyncInvokers.obj
 0001:000001b8       ??$launch@US_DDP@@P6A?AU1@XZ@@YA?AUS_DDP@@P6A?AU0@XZ@Z 00000001800011b8 f i libAsyncInvokers.obj
 0001:000001b8       ??$launch@US_DFP@@P6A?AU1@XZ@@YA?AUS_DFP@@P6A?AU0@XZ@Z 00000001800011b8 f i libAsyncInvokers.obj
 0001:000001b8       ??$launch@US_DIP@@P6A?AU1@XZ@@YA?AUS_DIP@@P6A?AU0@XZ@Z 00000001800011b8 f i libAsyncInvokers.obj
 0001:000001b8       ??$launch@US_DPD@@P6A?AU1@XZ@@YA?AUS_DPD@@P6A?AU0@XZ@Z 00000001800011b8 f i libAsyncInvokers.obj
 0001:000001b8       ??$launch@US_DPF@@P6A?AU1@XZ@@YA?AUS_DPF@@P6A?AU0@XZ@Z 00000001800011b8 f i libAsyncInvokers.obj
 0001:000001b8       ??$launch@US_DPI@@P6A?AU1@XZ@@YA?AUS_DPI@@P6A?AU0@XZ@Z 00000001800011b8 f i libAsyncInvokers.obj
 0001:000001b8       ??$launch@US_DPP@@P6A?AU1@XZ@@YA?AUS_DPP@@P6A?AU0@XZ@Z 00000001800011b8 f i libAsyncInvokers.obj
 0001:000001b8       ??$launch@US_FDP@@P6A?AU1@XZ@@YA?AUS_FDP@@P6A?AU0@XZ@Z 00000001800011b8 f i libAsyncInvokers.obj
 0001:000001b8       ??$launch@US_FPD@@P6A?AU1@XZ@@YA?AUS_FPD@@P6A?AU0@XZ@Z 00000001800011b8 f i libAsyncInvokers.obj
 0001:000001b8       ??$launch@US_FPF@@P6A?AU1@XZ@@YA?AUS_FPF@@P6A?AU0@XZ@Z 00000001800011b8 f i libAsyncInvokers.obj
 0001:000001b8       ??$launch@US_FPI@@P6A?AU1@XZ@@YA?AUS_FPI@@P6A?AU0@XZ@Z 00000001800011b8 f i libAsyncInvokers.obj
 0001:000001b8       ??$launch@US_FPP@@P6A?AU1@XZ@@YA?AUS_FPP@@P6A?AU0@XZ@Z 00000001800011b8 f i libAsyncInvokers.obj
 0001:000001b8       ??$launch@US_IDP@@P6A?AU1@XZ@@YA?AUS_IDP@@P6A?AU0@XZ@Z 00000001800011b8 f i libAsyncInvokers.obj
 0001:000001b8       ??$launch@US_IPD@@P6A?AU1@XZ@@YA?AUS_IPD@@P6A?AU0@XZ@Z 00000001800011b8 f i libAsyncInvokers.obj
 0001:000001b8       ??$launch@US_IPF@@P6A?AU1@XZ@@YA?AUS_IPF@@P6A?AU0@XZ@Z 00000001800011b8 f i libAsyncInvokers.obj
 0001:000001b8       ??$launch@US_IPI@@P6A?AU1@XZ@@YA?AUS_IPI@@P6A?AU0@XZ@Z 00000001800011b8 f i libAsyncInvokers.obj
 0001:000001b8       ??$launch@US_IPP@@P6A?AU1@XZ@@YA?AUS_IPP@@P6A?AU0@XZ@Z 00000001800011b8 f i libAsyncInvokers.obj
 0001:000001b8       ??$launch@US_PDD@@P6A?AU1@XZ@@YA?AUS_PDD@@P6A?AU0@XZ@Z 00000001800011b8 f i libAsyncInvokers.obj
 0001:000001b8       ??$launch@US_PDF@@P6A?AU1@XZ@@YA?AUS_PDF@@P6A?AU0@XZ@Z 00000001800011b8 f i libAsyncInvokers.obj
 0001:000001b8       ??$launch@US_PDI@@P6A?AU1@XZ@@YA?AUS_PDI@@P6A?AU0@XZ@Z 00000001800011b8 f i libAsyncInvokers.obj
 0001:000001b8       ??$launch@US_PDP@@P6A?AU1@XZ@@YA?AUS_PDP@@P6A?AU0@XZ@Z 00000001800011b8 f i libAsyncInvokers.obj
 0001:000001b8       ??$launch@US_PFD@@P6A?AU1@XZ@@YA?AUS_PFD@@P6A?AU0@XZ@Z 00000001800011b8 f i libAsyncInvokers.obj
 0001:000001b8       ??$launch@US_PFP@@P6A?AU1@XZ@@YA?AUS_PFP@@P6A?AU0@XZ@Z 00000001800011b8 f i libAsyncInvokers.obj
 0001:000001b8       ??$launch@US_PID@@P6A?AU1@XZ@@YA?AUS_PID@@P6A?AU0@XZ@Z 00000001800011b8 f i libAsyncInvokers.obj
 0001:000001b8       ??$launch@US_PIP@@P6A?AU1@XZ@@YA?AUS_PIP@@P6A?AU0@XZ@Z 00000001800011b8 f i libAsyncInvokers.obj
 0001:000001b8       ??$launch@US_PPD@@P6A?AU1@XZ@@YA?AUS_PPD@@P6A?AU0@XZ@Z 00000001800011b8 f i libAsyncInvokers.obj
 0001:000001b8       ??$launch@US_PPF@@P6A?AU1@XZ@@YA?AUS_PPF@@P6A?AU0@XZ@Z 00000001800011b8 f i libAsyncInvokers.obj
 0001:000001b8       ??$launch@US_PPI@@P6A?AU1@XZ@@YA?AUS_PPI@@P6A?AU0@XZ@Z 00000001800011b8 f i libAsyncInvokers.obj
 0001:000001b8       ??$launch@US_PPP@@P6A?AU1@XZ@@YA?AUS_PPP@@P6A?AU0@XZ@Z 00000001800011b8 f i libAsyncInvokers.obj
 0001:00000204       ??$launch@US_DP@@P6A?AU1@XZ@@YA?AUS_DP@@P6A?AU0@XZ@Z 0000000180001204 f i libAsyncInvokers.obj
 0001:00000204       ??$launch@US_FFP@@P6A?AU1@XZ@@YA?AUS_FFP@@P6A?AU0@XZ@Z 0000000180001204 f i libAsyncInvokers.obj
 0001:00000204       ??$launch@US_FIP@@P6A?AU1@XZ@@YA?AUS_FIP@@P6A?AU0@XZ@Z 0000000180001204 f i libAsyncInvokers.obj
 0001:00000204       ??$launch@US_FP@@P6A?AU1@XZ@@YA?AUS_FP@@P6A?AU0@XZ@Z 0000000180001204 f i libAsyncInvokers.obj
 0001:00000204       ??$launch@US_IFP@@P6A?AU1@XZ@@YA?AUS_IFP@@P6A?AU0@XZ@Z 0000000180001204 f i libAsyncInvokers.obj
 0001:00000204       ??$launch@US_IIP@@P6A?AU1@XZ@@YA?AUS_IIP@@P6A?AU0@XZ@Z 0000000180001204 f i libAsyncInvokers.obj
 0001:00000204       ??$launch@US_IP@@P6A?AU1@XZ@@YA?AUS_IP@@P6A?AU0@XZ@Z 0000000180001204 f i libAsyncInvokers.obj
 0001:00000204       ??$launch@US_PD@@P6A?AU1@XZ@@YA?AUS_PD@@P6A?AU0@XZ@Z 0000000180001204 f i libAsyncInvokers.obj
 0001:00000204       ??$launch@US_PF@@P6A?AU1@XZ@@YA?AUS_PF@@P6A?AU0@XZ@Z 0000000180001204 f i libAsyncInvokers.obj
 0001:00000204       ??$launch@US_PFF@@P6A?AU1@XZ@@YA?AUS_PFF@@P6A?AU0@XZ@Z 0000000180001204 f i libAsyncInvokers.obj
 0001:00000204       ??$launch@US_PFI@@P6A?AU1@XZ@@YA?AUS_PFI@@P6A?AU0@XZ@Z 0000000180001204 f i libAsyncInvokers.obj
 0001:00000204       ??$launch@US_PI@@P6A?AU1@XZ@@YA?AUS_PI@@P6A?AU0@XZ@Z 0000000180001204 f i libAsyncInvokers.obj
 0001:00000204       ??$launch@US_PIF@@P6A?AU1@XZ@@YA?AUS_PIF@@P6A?AU0@XZ@Z 0000000180001204 f i libAsyncInvokers.obj
 0001:00000204       ??$launch@US_PII@@P6A?AU1@XZ@@YA?AUS_PII@@P6A?AU0@XZ@Z 0000000180001204 f i libAsyncInvokers.obj
 0001:00000204       ??$launch@US_PP@@P6A?AU1@XZ@@YA?AUS_PP@@P6A?AU0@XZ@Z 0000000180001204 f i libAsyncInvokers.obj
 0001:00000248       ??$launch@US_F@@P6A?AU1@XZ@@YA?AUS_F@@P6A?AU0@XZ@Z 0000000180001248 f i libAsyncInvokers.obj
 0001:00000248       ??$launch@US_I@@P6A?AU1@XZ@@YA?AUS_I@@P6A?AU0@XZ@Z 0000000180001248 f i libAsyncInvokers.obj
 0001:00000278       ??$launch@US_FFF@@P6A?AU1@XZ@@YA?AUS_FFF@@P6A?AU0@XZ@Z 0000000180001278 f i libAsyncInvokers.obj
 0001:00000278       ??$launch@US_FFI@@P6A?AU1@XZ@@YA?AUS_FFI@@P6A?AU0@XZ@Z 0000000180001278 f i libAsyncInvokers.obj
 0001:00000278       ??$launch@US_FIF@@P6A?AU1@XZ@@YA?AUS_FIF@@P6A?AU0@XZ@Z 0000000180001278 f i libAsyncInvokers.obj
 0001:00000278       ??$launch@US_FII@@P6A?AU1@XZ@@YA?AUS_FII@@P6A?AU0@XZ@Z 0000000180001278 f i libAsyncInvokers.obj
 0001:00000278       ??$launch@US_IFF@@P6A?AU1@XZ@@YA?AUS_IFF@@P6A?AU0@XZ@Z 0000000180001278 f i libAsyncInvokers.obj
 0001:00000278       ??$launch@US_IFI@@P6A?AU1@XZ@@YA?AUS_IFI@@P6A?AU0@XZ@Z 0000000180001278 f i libAsyncInvokers.obj
 0001:00000278       ??$launch@US_IIF@@P6A?AU1@XZ@@YA?AUS_IIF@@P6A?AU0@XZ@Z 0000000180001278 f i libAsyncInvokers.obj
 0001:00000278       ??$launch@US_III@@P6A?AU1@XZ@@YA?AUS_III@@P6A?AU0@XZ@Z 0000000180001278 f i libAsyncInvokers.obj
 0001:000002e0       ??$launch_v@P6AXXZ@@YAXP6AXXZ@Z 00000001800012e0 f i libAsyncInvokers.obj
 0001:00000300       ??$proc@HP6AHXZ@@YAXPEAX@Z 0000000180001300 f i libAsyncInvokers.obj
 0001:00000328       ??$proc@MP6AMXZ@@YAXPEAX@Z 0000000180001328 f i libAsyncInvokers.obj
 0001:00000354       ??$proc@NP6ANXZ@@YAXPEAX@Z 0000000180001354 f i libAsyncInvokers.obj
 0001:00000380       ??$proc@PEAXP6APEAXXZ@@YAXPEAX@Z 0000000180001380 f i libAsyncInvokers.obj
 0001:000003a8       ??$proc@US_D@@P6A?AU1@XZ@@YAXPEAX@Z 00000001800013a8 f i libAsyncInvokers.obj
 0001:000003a8       ??$proc@US_FF@@P6A?AU1@XZ@@YAXPEAX@Z 00000001800013a8 f i libAsyncInvokers.obj
 0001:000003a8       ??$proc@US_FI@@P6A?AU1@XZ@@YAXPEAX@Z 00000001800013a8 f i libAsyncInvokers.obj
 0001:000003a8       ??$proc@US_IF@@P6A?AU1@XZ@@YAXPEAX@Z 00000001800013a8 f i libAsyncInvokers.obj
 0001:000003a8       ??$proc@US_II@@P6A?AU1@XZ@@YAXPEAX@Z 00000001800013a8 f i libAsyncInvokers.obj
 0001:000003a8       ??$proc@US_P@@P6A?AU1@XZ@@YAXPEAX@Z 00000001800013a8 f i libAsyncInvokers.obj
 0001:000003dc       ??$proc@US_DD@@P6A?AU1@XZ@@YAXPEAX@Z 00000001800013dc f i libAsyncInvokers.obj
 0001:000003dc       ??$proc@US_DF@@P6A?AU1@XZ@@YAXPEAX@Z 00000001800013dc f i libAsyncInvokers.obj
 0001:000003dc       ??$proc@US_DFF@@P6A?AU1@XZ@@YAXPEAX@Z 00000001800013dc f i libAsyncInvokers.obj
 0001:000003dc       ??$proc@US_DFI@@P6A?AU1@XZ@@YAXPEAX@Z 00000001800013dc f i libAsyncInvokers.obj
 0001:000003dc       ??$proc@US_DI@@P6A?AU1@XZ@@YAXPEAX@Z 00000001800013dc f i libAsyncInvokers.obj
 0001:000003dc       ??$proc@US_DIF@@P6A?AU1@XZ@@YAXPEAX@Z 00000001800013dc f i libAsyncInvokers.obj
 0001:000003dc       ??$proc@US_DII@@P6A?AU1@XZ@@YAXPEAX@Z 00000001800013dc f i libAsyncInvokers.obj
 0001:000003dc       ??$proc@US_FD@@P6A?AU1@XZ@@YAXPEAX@Z 00000001800013dc f i libAsyncInvokers.obj
 0001:000003dc       ??$proc@US_FFD@@P6A?AU1@XZ@@YAXPEAX@Z 00000001800013dc f i libAsyncInvokers.obj
 0001:000003dc       ??$proc@US_FID@@P6A?AU1@XZ@@YAXPEAX@Z 00000001800013dc f i libAsyncInvokers.obj
 0001:000003dc       ??$proc@US_ID@@P6A?AU1@XZ@@YAXPEAX@Z 00000001800013dc f i libAsyncInvokers.obj
 0001:000003dc       ??$proc@US_IFD@@P6A?AU1@XZ@@YAXPEAX@Z 00000001800013dc f i libAsyncInvokers.obj
 0001:000003dc       ??$proc@US_IID@@P6A?AU1@XZ@@YAXPEAX@Z 00000001800013dc f i libAsyncInvokers.obj
 0001:00000434       ??$proc@US_DDD@@P6A?AU1@XZ@@YAXPEAX@Z 0000000180001434 f i libAsyncInvokers.obj
 0001:00000434       ??$proc@US_DDF@@P6A?AU1@XZ@@YAXPEAX@Z 0000000180001434 f i libAsyncInvokers.obj
 0001:00000434       ??$proc@US_DDI@@P6A?AU1@XZ@@YAXPEAX@Z 0000000180001434 f i libAsyncInvokers.obj
 0001:00000434       ??$proc@US_DFD@@P6A?AU1@XZ@@YAXPEAX@Z 0000000180001434 f i libAsyncInvokers.obj
 0001:00000434       ??$proc@US_DID@@P6A?AU1@XZ@@YAXPEAX@Z 0000000180001434 f i libAsyncInvokers.obj
 0001:00000434       ??$proc@US_FDD@@P6A?AU1@XZ@@YAXPEAX@Z 0000000180001434 f i libAsyncInvokers.obj
 0001:00000434       ??$proc@US_FDF@@P6A?AU1@XZ@@YAXPEAX@Z 0000000180001434 f i libAsyncInvokers.obj
 0001:00000434       ??$proc@US_FDI@@P6A?AU1@XZ@@YAXPEAX@Z 0000000180001434 f i libAsyncInvokers.obj
 0001:00000434       ??$proc@US_IDD@@P6A?AU1@XZ@@YAXPEAX@Z 0000000180001434 f i libAsyncInvokers.obj
 0001:00000434       ??$proc@US_IDF@@P6A?AU1@XZ@@YAXPEAX@Z 0000000180001434 f i libAsyncInvokers.obj
 0001:00000434       ??$proc@US_IDI@@P6A?AU1@XZ@@YAXPEAX@Z 0000000180001434 f i libAsyncInvokers.obj
 0001:000004a8       ??$proc@US_DDP@@P6A?AU1@XZ@@YAXPEAX@Z 00000001800014a8 f i libAsyncInvokers.obj
 0001:000004a8       ??$proc@US_DFP@@P6A?AU1@XZ@@YAXPEAX@Z 00000001800014a8 f i libAsyncInvokers.obj
 0001:000004a8       ??$proc@US_DIP@@P6A?AU1@XZ@@YAXPEAX@Z 00000001800014a8 f i libAsyncInvokers.obj
 0001:000004a8       ??$proc@US_DPD@@P6A?AU1@XZ@@YAXPEAX@Z 00000001800014a8 f i libAsyncInvokers.obj
 0001:000004a8       ??$proc@US_DPF@@P6A?AU1@XZ@@YAXPEAX@Z 00000001800014a8 f i libAsyncInvokers.obj
 0001:000004a8       ??$proc@US_DPI@@P6A?AU1@XZ@@YAXPEAX@Z 00000001800014a8 f i libAsyncInvokers.obj
 0001:000004a8       ??$proc@US_DPP@@P6A?AU1@XZ@@YAXPEAX@Z 00000001800014a8 f i libAsyncInvokers.obj
 0001:000004a8       ??$proc@US_FDP@@P6A?AU1@XZ@@YAXPEAX@Z 00000001800014a8 f i libAsyncInvokers.obj
 0001:000004a8       ??$proc@US_FPD@@P6A?AU1@XZ@@YAXPEAX@Z 00000001800014a8 f i libAsyncInvokers.obj
 0001:000004a8       ??$proc@US_FPF@@P6A?AU1@XZ@@YAXPEAX@Z 00000001800014a8 f i libAsyncInvokers.obj
 0001:000004a8       ??$proc@US_FPI@@P6A?AU1@XZ@@YAXPEAX@Z 00000001800014a8 f i libAsyncInvokers.obj
 0001:000004a8       ??$proc@US_FPP@@P6A?AU1@XZ@@YAXPEAX@Z 00000001800014a8 f i libAsyncInvokers.obj
 0001:000004a8       ??$proc@US_IDP@@P6A?AU1@XZ@@YAXPEAX@Z 00000001800014a8 f i libAsyncInvokers.obj
 0001:000004a8       ??$proc@US_IPD@@P6A?AU1@XZ@@YAXPEAX@Z 00000001800014a8 f i libAsyncInvokers.obj
 0001:000004a8       ??$proc@US_IPF@@P6A?AU1@XZ@@YAXPEAX@Z 00000001800014a8 f i libAsyncInvokers.obj
 0001:000004a8       ??$proc@US_IPI@@P6A?AU1@XZ@@YAXPEAX@Z 00000001800014a8 f i libAsyncInvokers.obj
 0001:000004a8       ??$proc@US_IPP@@P6A?AU1@XZ@@YAXPEAX@Z 00000001800014a8 f i libAsyncInvokers.obj
 0001:000004a8       ??$proc@US_PDD@@P6A?AU1@XZ@@YAXPEAX@Z 00000001800014a8 f i libAsyncInvokers.obj
 0001:000004a8       ??$proc@US_PDF@@P6A?AU1@XZ@@YAXPEAX@Z 00000001800014a8 f i libAsyncInvokers.obj
 0001:000004a8       ??$proc@US_PDI@@P6A?AU1@XZ@@YAXPEAX@Z 00000001800014a8 f i libAsyncInvokers.obj
 0001:000004a8       ??$proc@US_PDP@@P6A?AU1@XZ@@YAXPEAX@Z 00000001800014a8 f i libAsyncInvokers.obj
 0001:000004a8       ??$proc@US_PFD@@P6A?AU1@XZ@@YAXPEAX@Z 00000001800014a8 f i libAsyncInvokers.obj
 0001:000004a8       ??$proc@US_PFP@@P6A?AU1@XZ@@YAXPEAX@Z 00000001800014a8 f i libAsyncInvokers.obj
 0001:000004a8       ??$proc@US_PID@@P6A?AU1@XZ@@YAXPEAX@Z 00000001800014a8 f i libAsyncInvokers.obj
 0001:000004a8       ??$proc@US_PIP@@P6A?AU1@XZ@@YAXPEAX@Z 00000001800014a8 f i libAsyncInvokers.obj
 0001:000004a8       ??$proc@US_PPD@@P6A?AU1@XZ@@YAXPEAX@Z 00000001800014a8 f i libAsyncInvokers.obj
 0001:000004a8       ??$proc@US_PPF@@P6A?AU1@XZ@@YAXPEAX@Z 00000001800014a8 f i libAsyncInvokers.obj
 0001:000004a8       ??$proc@US_PPI@@P6A?AU1@XZ@@YAXPEAX@Z 00000001800014a8 f i libAsyncInvokers.obj
 0001:000004a8       ??$proc@US_PPP@@P6A?AU1@XZ@@YAXPEAX@Z 00000001800014a8 f i libAsyncInvokers.obj
 0001:00000500       ??$proc@US_DP@@P6A?AU1@XZ@@YAXPEAX@Z 0000000180001500 f i libAsyncInvokers.obj
 0001:00000500       ??$proc@US_FFP@@P6A?AU1@XZ@@YAXPEAX@Z 0000000180001500 f i libAsyncInvokers.obj
 0001:00000500       ??$proc@US_FIP@@P6A?AU1@XZ@@YAXPEAX@Z 0000000180001500 f i libAsyncInvokers.obj
 0001:00000500       ??$proc@US_FP@@P6A?AU1@XZ@@YAXPEAX@Z 0000000180001500 f i libAsyncInvokers.obj
 0001:00000500       ??$proc@US_IFP@@P6A?AU1@XZ@@YAXPEAX@Z 0000000180001500 f i libAsyncInvokers.obj
 0001:00000500       ??$proc@US_IIP@@P6A?AU1@XZ@@YAXPEAX@Z 0000000180001500 f i libAsyncInvokers.obj
 0001:00000500       ??$proc@US_IP@@P6A?AU1@XZ@@YAXPEAX@Z 0000000180001500 f i libAsyncInvokers.obj
 0001:00000500       ??$proc@US_PD@@P6A?AU1@XZ@@YAXPEAX@Z 0000000180001500 f i libAsyncInvokers.obj
 0001:00000500       ??$proc@US_PF@@P6A?AU1@XZ@@YAXPEAX@Z 0000000180001500 f i libAsyncInvokers.obj
 0001:00000500       ??$proc@US_PFF@@P6A?AU1@XZ@@YAXPEAX@Z 0000000180001500 f i libAsyncInvokers.obj
 0001:00000500       ??$proc@US_PFI@@P6A?AU1@XZ@@YAXPEAX@Z 0000000180001500 f i libAsyncInvokers.obj
 0001:00000500       ??$proc@US_PI@@P6A?AU1@XZ@@YAXPEAX@Z 0000000180001500 f i libAsyncInvokers.obj
 0001:00000500       ??$proc@US_PIF@@P6A?AU1@XZ@@YAXPEAX@Z 0000000180001500 f i libAsyncInvokers.obj
 0001:00000500       ??$proc@US_PII@@P6A?AU1@XZ@@YAXPEAX@Z 0000000180001500 f i libAsyncInvokers.obj
 0001:00000500       ??$proc@US_PP@@P6A?AU1@XZ@@YAXPEAX@Z 0000000180001500 f i libAsyncInvokers.obj
 0001:0000053c       ??$proc@US_F@@P6A?AU1@XZ@@YAXPEAX@Z 000000018000153c f i libAsyncInvokers.obj
 0001:0000053c       ??$proc@US_I@@P6A?AU1@XZ@@YAXPEAX@Z 000000018000153c f i libAsyncInvokers.obj
 0001:0000056c       ??$proc@US_FFF@@P6A?AU1@XZ@@YAXPEAX@Z 000000018000156c f i libAsyncInvokers.obj
 0001:0000056c       ??$proc@US_FFI@@P6A?AU1@XZ@@YAXPEAX@Z 000000018000156c f i libAsyncInvokers.obj
 0001:0000056c       ??$proc@US_FIF@@P6A?AU1@XZ@@YAXPEAX@Z 000000018000156c f i libAsyncInvokers.obj
 0001:0000056c       ??$proc@US_FII@@P6A?AU1@XZ@@YAXPEAX@Z 000000018000156c f i libAsyncInvokers.obj
 0001:0000056c       ??$proc@US_IFF@@P6A?AU1@XZ@@YAXPEAX@Z 000000018000156c f i libAsyncInvokers.obj
 0001:0000056c       ??$proc@US_IFI@@P6A?AU1@XZ@@YAXPEAX@Z 000000018000156c f i libAsyncInvokers.obj
 0001:0000056c       ??$proc@US_IIF@@P6A?AU1@XZ@@YAXPEAX@Z 000000018000156c f i libAsyncInvokers.obj
 0001:0000056c       ??$proc@US_III@@P6A?AU1@XZ@@YAXPEAX@Z 000000018000156c f i libAsyncInvokers.obj
 0001:000005dc       ??$proc_v@P6AXXZ@@YAXPEAX@Z 00000001800015dc f i libAsyncInvokers.obj
 0001:000005f0       call_async_D               00000001800015f0 f   libAsyncInvokers.obj
 0001:00000608       call_async_F               0000000180001608 f   libAsyncInvokers.obj
 0001:00000620       call_async_I               0000000180001620 f   libAsyncInvokers.obj
 0001:00000638       call_async_P               0000000180001638 f   libAsyncInvokers.obj
 0001:00000650       call_async_S_D             0000000180001650 f   libAsyncInvokers.obj
 0001:00000650       call_async_S_FF            0000000180001650 f   libAsyncInvokers.obj
 0001:00000650       call_async_S_FI            0000000180001650 f   libAsyncInvokers.obj
 0001:00000650       call_async_S_IF            0000000180001650 f   libAsyncInvokers.obj
 0001:00000650       call_async_S_II            0000000180001650 f   libAsyncInvokers.obj
 0001:00000650       call_async_S_P             0000000180001650 f   libAsyncInvokers.obj
 0001:00000674       call_async_S_DD            0000000180001674 f   libAsyncInvokers.obj
 0001:00000674       call_async_S_DF            0000000180001674 f   libAsyncInvokers.obj
 0001:00000674       call_async_S_DFF           0000000180001674 f   libAsyncInvokers.obj
 0001:00000674       call_async_S_DFI           0000000180001674 f   libAsyncInvokers.obj
 0001:00000674       call_async_S_DI            0000000180001674 f   libAsyncInvokers.obj
 0001:00000674       call_async_S_DIF           0000000180001674 f   libAsyncInvokers.obj
 0001:00000674       call_async_S_DII           0000000180001674 f   libAsyncInvokers.obj
 0001:00000674       call_async_S_FD            0000000180001674 f   libAsyncInvokers.obj
 0001:00000674       call_async_S_FFD           0000000180001674 f   libAsyncInvokers.obj
 0001:00000674       call_async_S_FID           0000000180001674 f   libAsyncInvokers.obj
 0001:00000674       call_async_S_ID            0000000180001674 f   libAsyncInvokers.obj
 0001:00000674       call_async_S_IFD           0000000180001674 f   libAsyncInvokers.obj
 0001:00000674       call_async_S_IID           0000000180001674 f   libAsyncInvokers.obj
 0001:000006d0       call_async_S_DDD           00000001800016d0 f   libAsyncInvokers.obj
 0001:000006d0       call_async_S_DDF           00000001800016d0 f   libAsyncInvokers.obj
 0001:000006d0       call_async_S_DDI           00000001800016d0 f   libAsyncInvokers.obj
 0001:000006d0       call_async_S_DFD           00000001800016d0 f   libAsyncInvokers.obj
 0001:000006d0       call_async_S_DID           00000001800016d0 f   libAsyncInvokers.obj
 0001:000006d0       call_async_S_FDD           00000001800016d0 f   libAsyncInvokers.obj
 0001:000006d0       call_async_S_FDF           00000001800016d0 f   libAsyncInvokers.obj
 0001:000006d0       call_async_S_FDI           00000001800016d0 f   libAsyncInvokers.obj
 0001:000006d0       call_async_S_IDD           00000001800016d0 f   libAsyncInvokers.obj
 0001:000006d0       call_async_S_IDF           00000001800016d0 f   libAsyncInvokers.obj
 0001:000006d0       call_async_S_IDI           00000001800016d0 f   libAsyncInvokers.obj
 0001:00000748       call_async_S_DDP           0000000180001748 f   libAsyncInvokers.obj
 0001:00000748       call_async_S_DFP           0000000180001748 f   libAsyncInvokers.obj
 0001:00000748       call_async_S_DIP           0000000180001748 f   libAsyncInvokers.obj
 0001:00000748       call_async_S_DPD           0000000180001748 f   libAsyncInvokers.obj
 0001:00000748       call_async_S_DPF           0000000180001748 f   libAsyncInvokers.obj
 0001:00000748       call_async_S_DPI           0000000180001748 f   libAsyncInvokers.obj
 0001:00000748       call_async_S_DPP           0000000180001748 f   libAsyncInvokers.obj
 0001:00000748       call_async_S_FDP           0000000180001748 f   libAsyncInvokers.obj
 0001:00000748       call_async_S_FPD           0000000180001748 f   libAsyncInvokers.obj
 0001:00000748       call_async_S_FPF           0000000180001748 f   libAsyncInvokers.obj
 0001:00000748       call_async_S_FPI           0000000180001748 f   libAsyncInvokers.obj
 0001:00000748       call_async_S_FPP           0000000180001748 f   libAsyncInvokers.obj
 0001:00000748       call_async_S_IDP           0000000180001748 f   libAsyncInvokers.obj
 0001:00000748       call_async_S_IPD           0000000180001748 f   libAsyncInvokers.obj
 0001:00000748       call_async_S_IPF           0000000180001748 f   libAsyncInvokers.obj
 0001:00000748       call_async_S_IPI           0000000180001748 f   libAsyncInvokers.obj
 0001:00000748       call_async_S_IPP           0000000180001748 f   libAsyncInvokers.obj
 0001:00000748       call_async_S_PDD           0000000180001748 f   libAsyncInvokers.obj
 0001:00000748       call_async_S_PDF           0000000180001748 f   libAsyncInvokers.obj
 0001:00000748       call_async_S_PDI           0000000180001748 f   libAsyncInvokers.obj
 0001:00000748       call_async_S_PDP           0000000180001748 f   libAsyncInvokers.obj
 0001:00000748       call_async_S_PFD           0000000180001748 f   libAsyncInvokers.obj
 0001:00000748       call_async_S_PFP           0000000180001748 f   libAsyncInvokers.obj
 0001:00000748       call_async_S_PID           0000000180001748 f   libAsyncInvokers.obj
 0001:00000748       call_async_S_PIP           0000000180001748 f   libAsyncInvokers.obj
 0001:00000748       call_async_S_PPD           0000000180001748 f   libAsyncInvokers.obj
 0001:00000748       call_async_S_PPF           0000000180001748 f   libAsyncInvokers.obj
 0001:00000748       call_async_S_PPI           0000000180001748 f   libAsyncInvokers.obj
 0001:00000748       call_async_S_PPP           0000000180001748 f   libAsyncInvokers.obj
 0001:0000079c       call_async_S_DP            000000018000179c f   libAsyncInvokers.obj
 0001:0000079c       call_async_S_FFP           000000018000179c f   libAsyncInvokers.obj
 0001:0000079c       call_async_S_FIP           000000018000179c f   libAsyncInvokers.obj
 0001:0000079c       call_async_S_FP            000000018000179c f   libAsyncInvokers.obj
 0001:0000079c       call_async_S_IFP           000000018000179c f   libAsyncInvokers.obj
 0001:0000079c       call_async_S_IIP           000000018000179c f   libAsyncInvokers.obj
 0001:0000079c       call_async_S_IP            000000018000179c f   libAsyncInvokers.obj
 0001:0000079c       call_async_S_PD            000000018000179c f   libAsyncInvokers.obj
 0001:0000079c       call_async_S_PF            000000018000179c f   libAsyncInvokers.obj
 0001:0000079c       call_async_S_PFF           000000018000179c f   libAsyncInvokers.obj
 0001:0000079c       call_async_S_PFI           000000018000179c f   libAsyncInvokers.obj
 0001:0000079c       call_async_S_PI            000000018000179c f   libAsyncInvokers.obj
 0001:0000079c       call_async_S_PIF           000000018000179c f   libAsyncInvokers.obj
 0001:0000079c       call_async_S_PII           000000018000179c f   libAsyncInvokers.obj
 0001:0000079c       call_async_S_PP            000000018000179c f   libAsyncInvokers.obj
 0001:000007dc       call_async_S_F             00000001800017dc f   libAsyncInvokers.obj
 0001:000007dc       call_async_S_I             00000001800017dc f   libAsyncInvokers.obj
 0001:000007fc       call_async_S_FFF           00000001800017fc f   libAsyncInvokers.obj
 0001:000007fc       call_async_S_FFI           00000001800017fc f   libAsyncInvokers.obj
 0001:000007fc       call_async_S_FIF           00000001800017fc f   libAsyncInvokers.obj
 0001:000007fc       call_async_S_FII           00000001800017fc f   libAsyncInvokers.obj
 0001:000007fc       call_async_S_IFF           00000001800017fc f   libAsyncInvokers.obj
 0001:000007fc       call_async_S_IFI           00000001800017fc f   libAsyncInvokers.obj
 0001:000007fc       call_async_S_IIF           00000001800017fc f   libAsyncInvokers.obj
 0001:000007fc       call_async_S_III           00000001800017fc f   libAsyncInvokers.obj
 0001:0000086c       call_async_V               000000018000186c f   libAsyncInvokers.obj
 0001:000008b4       procedure                  00000001800018b4 f   libAsyncInvokers.obj
 0001:000008c8       run_in_new_thread_and_join 00000001800018c8 f   libAsyncInvokers.obj
 0001:0000093c       __GSHandlerCheck           000000018000193c f   MSVCRT:gshandler.obj
 0001:0000095c       __GSHandlerCheckCommon     000000018000195c f   MSVCRT:gshandler.obj
 0001:000009d0       __security_check_cookie    00000001800019d0 f   MSVCRT:amdsecgs.obj
 0001:00000d10       _DllMainCRTStartup         0000000180001d10 f   MSVCRT:dll_dllmain.obj
 0001:00000d50       __raise_securityfailure    0000000180001d50 f   MSVCRT:gs_report.obj
 0001:00000d84       __report_gsfailure         0000000180001d84 f   MSVCRT:gs_report.obj
 0001:00000ecc       __security_init_cookie     0000000180001ecc f   MSVCRT:gs_support.obj
 0001:00000f78       DllMain                    0000000180001f78 f   MSVCRT:dll_dllmain_stub.obj
 0001:00000f9c       ?__scrt_initialize_type_info@@YAXXZ 0000000180001f9c f   MSVCRT:tncleanup.obj
 0001:00000fac       ?__scrt_uninitialize_type_info@@YAXXZ 0000000180001fac f   MSVCRT:tncleanup.obj
 0001:00000fb8       __local_stdio_printf_options 0000000180001fb8 f i MSVCRT:default_local_stdio_options.obj
 0001:00000fc0       __local_stdio_scanf_options 0000000180001fc0 f i MSVCRT:default_local_stdio_options.obj
 0001:00000fc8       __scrt_initialize_default_local_stdio_options 0000000180001fc8 f   MSVCRT:default_local_stdio_options.obj
 0001:00000fe4       __scrt_acquire_startup_lock 0000000180001fe4 f   MSVCRT:utility.obj
 0001:00001020       __scrt_dllmain_after_initialize_c 0000000180002020 f   MSVCRT:utility.obj
 0001:00001054       __scrt_dllmain_before_initialize_c 0000000180002054 f   MSVCRT:utility.obj
 0001:0000106c       __scrt_dllmain_crt_thread_attach 000000018000206c f   MSVCRT:utility.obj
 0001:00001094       __scrt_dllmain_crt_thread_detach 0000000180002094 f   MSVCRT:utility.obj
 0001:000010ac       __scrt_dllmain_exception_filter 00000001800020ac f   MSVCRT:utility.obj
 0001:0000110c       __scrt_dllmain_uninitialize_c 000000018000210c f   MSVCRT:utility.obj
 0001:0000113c       __scrt_dllmain_uninitialize_critical 000000018000213c f   MSVCRT:utility.obj
 0001:00001150       __scrt_initialize_crt      0000000180002150 f   MSVCRT:utility.obj
 0001:0000119c       __scrt_initialize_onexit_tables 000000018000219c f   MSVCRT:utility.obj
 0001:00001228       __scrt_is_nonwritable_in_current_image 0000000180002228 f   MSVCRT:utility.obj
 0001:000012c0       __scrt_release_startup_lock 00000001800022c0 f   MSVCRT:utility.obj
 0001:000012e4       __scrt_uninitialize_crt    00000001800022e4 f   MSVCRT:utility.obj
 0001:00001310       __scrt_get_dyn_tls_init_callback 0000000180002310 f   MSVCRT:dyn_tls_init.obj
 0001:00001318       __crt_debugger_hook        0000000180002318 f   MSVCRT:utility_desktop.obj
 0001:00001320       __scrt_fastfail            0000000180002320 f   MSVCRT:utility_desktop.obj
 0001:0000146c       _RTC_Initialize            000000018000246c f   MSVCRT:initsect.obj
 0001:000014a8       _RTC_Terminate             00000001800024a8 f   MSVCRT:initsect.obj
 0001:000014e4       _guard_check_icall_nop     00000001800024e4 f i MSVCRT:guard_support.obj
 0001:000014e8       __isa_available_init       00000001800024e8 f   MSVCRT:cpu_disp.obj
 0001:00001694       _get_startup_argv_mode     0000000180002694 f   MSVCRT:argv_mode.obj
 0001:0000169c       __scrt_is_ucrt_dll_in_use  000000018000269c f   MSVCRT:ucrt_detection.obj
 0001:000016b0       __C_specific_handler       00000001800026b0 f   vcruntime:VCRUNTIME140.dll
 0001:000016b6       __std_type_info_destroy_list 00000001800026b6 f   vcruntime:VCRUNTIME140.dll
 0001:000016bc       memset                     00000001800026bc f   vcruntime:VCRUNTIME140.dll
 0001:000016c2       _initterm                  00000001800026c2 f   ucrt:api-ms-win-crt-runtime-l1-1-0.dll
 0001:000016c8       _initterm_e                00000001800026c8 f   ucrt:api-ms-win-crt-runtime-l1-1-0.dll
 0001:000016ce       _seh_filter_dll            00000001800026ce f   ucrt:api-ms-win-crt-runtime-l1-1-0.dll
 0001:000016d4       _configure_narrow_argv     00000001800026d4 f   ucrt:api-ms-win-crt-runtime-l1-1-0.dll
 0001:000016da       _initialize_narrow_environment 00000001800026da f   ucrt:api-ms-win-crt-runtime-l1-1-0.dll
 0001:000016e0       _initialize_onexit_table   00000001800026e0 f   ucrt:api-ms-win-crt-runtime-l1-1-0.dll
 0001:000016e6       _execute_onexit_table      00000001800026e6 f   ucrt:api-ms-win-crt-runtime-l1-1-0.dll
 0001:000016ec       _cexit                     00000001800026ec f   ucrt:api-ms-win-crt-runtime-l1-1-0.dll
 0001:000016f4       __acrt_initialize          00000001800026f4 f   MSVCRT:ucrt_stubs.obj
 0001:000016f4       __acrt_thread_attach       00000001800026f4 f   MSVCRT:ucrt_stubs.obj
 0001:000016f4       __acrt_thread_detach       00000001800026f4 f   MSVCRT:ucrt_stubs.obj
 0001:000016f4       __acrt_uninitialize        00000001800026f4 f   MSVCRT:ucrt_stubs.obj
 0001:000016f4       __acrt_uninitialize_critical 00000001800026f4 f   MSVCRT:ucrt_stubs.obj
 0001:000016f4       __scrt_stub_for_acrt_initialize 00000001800026f4 f   MSVCRT:ucrt_stubs.obj
 0001:000016f4       __scrt_stub_for_acrt_thread_attach 00000001800026f4 f   MSVCRT:ucrt_stubs.obj
 0001:000016f4       __scrt_stub_for_acrt_thread_detach 00000001800026f4 f   MSVCRT:ucrt_stubs.obj
 0001:000016f4       __scrt_stub_for_acrt_uninitialize 00000001800026f4 f   MSVCRT:ucrt_stubs.obj
 0001:000016f4       __scrt_stub_for_acrt_uninitialize_critical 00000001800026f4 f   MSVCRT:ucrt_stubs.obj
 0001:000016f4       __vcrt_initialize          00000001800026f4 f   MSVCRT:ucrt_stubs.obj
 0001:000016f4       __vcrt_thread_attach       00000001800026f4 f   MSVCRT:ucrt_stubs.obj
 0001:000016f4       __vcrt_thread_detach       00000001800026f4 f   MSVCRT:ucrt_stubs.obj
 0001:000016f4       __vcrt_uninitialize        00000001800026f4 f   MSVCRT:ucrt_stubs.obj
 0001:000016f4       __vcrt_uninitialize_critical 00000001800026f4 f   MSVCRT:ucrt_stubs.obj
 0001:000016f8       __scrt_stub_for_is_c_termination_complete 00000001800026f8 f   MSVCRT:ucrt_stubs.obj
 0001:000016f8       _is_c_termination_complete 00000001800026f8 f   MSVCRT:ucrt_stubs.obj
 0001:000016fb       memcpy                     00000001800026fb f   vcruntime:VCRUNTIME140.dll
 0001:00001720       _guard_dispatch_icall_nop  0000000180002720 f   MSVCRT:guard_dispatch.obj
 0001:00001740       _guard_xfg_dispatch_icall_nop 0000000180002740 f   MSVCRT:guard_xfg_dispatch.obj
 0002:00000000       __imp_GetLastError         0000000180003000     kernel32:KERNEL32.dll
 0002:00000008       __imp_WaitForSingleObject  0000000180003008     kernel32:KERNEL32.dll
 0002:00000010       __imp_CreateThread         0000000180003010     kernel32:KERNEL32.dll
 0002:00000018       __imp_RtlCaptureContext    0000000180003018     kernel32:KERNEL32.dll
 0002:00000020       __imp_RtlLookupFunctionEntry 0000000180003020     kernel32:KERNEL32.dll
 0002:00000028       __imp_RtlVirtualUnwind     0000000180003028     kernel32:KERNEL32.dll
 0002:00000030       __imp_UnhandledExceptionFilter 0000000180003030     kernel32:KERNEL32.dll
 0002:00000038       __imp_SetUnhandledExceptionFilter 0000000180003038     kernel32:KERNEL32.dll
 0002:00000040       __imp_GetCurrentProcess    0000000180003040     kernel32:KERNEL32.dll
 0002:00000048       __imp_TerminateProcess     0000000180003048     kernel32:KERNEL32.dll
 0002:00000050       __imp_IsProcessorFeaturePresent 0000000180003050     kernel32:KERNEL32.dll
 0002:00000058       __imp_QueryPerformanceCounter 0000000180003058     kernel32:KERNEL32.dll
 0002:00000060       __imp_GetCurrentProcessId  0000000180003060     kernel32:KERNEL32.dll
 0002:00000068       __imp_GetCurrentThreadId   0000000180003068     kernel32:KERNEL32.dll
 0002:00000070       __imp_GetSystemTimeAsFileTime 0000000180003070     kernel32:KERNEL32.dll
 0002:00000078       __imp_DisableThreadLibraryCalls 0000000180003078     kernel32:KERNEL32.dll
 0002:00000080       __imp_InitializeSListHead  0000000180003080     kernel32:KERNEL32.dll
 0002:00000088       __imp_IsDebuggerPresent    0000000180003088     kernel32:KERNEL32.dll
 0002:00000090       \177KERNEL32_NULL_THUNK_DATA 0000000180003090     kernel32:KERNEL32.dll
 0002:00000098       __imp___C_specific_handler 0000000180003098     vcruntime:VCRUNTIME140.dll
 0002:000000a0       __imp___std_type_info_destroy_list 00000001800030a0     vcruntime:VCRUNTIME140.dll
 0002:000000a8       __imp_memset               00000001800030a8     vcruntime:VCRUNTIME140.dll
 0002:000000b0       __imp_memcpy               00000001800030b0     vcruntime:VCRUNTIME140.dll
 0002:000000b8       \177VCRUNTIME140_NULL_THUNK_DATA 00000001800030b8     vcruntime:VCRUNTIME140.dll
 0002:000000c0       __imp__initterm            00000001800030c0     ucrt:api-ms-win-crt-runtime-l1-1-0.dll
 0002:000000c8       __imp__initterm_e          00000001800030c8     ucrt:api-ms-win-crt-runtime-l1-1-0.dll
 0002:000000d0       __imp__seh_filter_dll      00000001800030d0     ucrt:api-ms-win-crt-runtime-l1-1-0.dll
 0002:000000d8       __imp__configure_narrow_argv 00000001800030d8     ucrt:api-ms-win-crt-runtime-l1-1-0.dll
 0002:000000e0       __imp__initialize_narrow_environment 00000001800030e0     ucrt:api-ms-win-crt-runtime-l1-1-0.dll
 0002:000000e8       __imp_exit                 00000001800030e8     ucrt:api-ms-win-crt-runtime-l1-1-0.dll
 0002:000000f0       __imp__initialize_onexit_table 00000001800030f0     ucrt:api-ms-win-crt-runtime-l1-1-0.dll
 0002:000000f8       __imp__execute_onexit_table 00000001800030f8     ucrt:api-ms-win-crt-runtime-l1-1-0.dll
 0002:00000100       __imp__cexit               0000000180003100     ucrt:api-ms-win-crt-runtime-l1-1-0.dll
 0002:00000108       \177api-ms-win-crt-runtime-l1-1-0_NULL_THUNK_DATA 0000000180003108     ucrt:api-ms-win-crt-runtime-l1-1-0.dll
 0002:00000110       __imp___acrt_iob_func      0000000180003110     ucrt:api-ms-win-crt-stdio-l1-1-0.dll
 0002:00000118       __imp_fputs                0000000180003118     ucrt:api-ms-win-crt-stdio-l1-1-0.dll
 0002:00000120       \177api-ms-win-crt-stdio-l1-1-0_NULL_THUNK_DATA 0000000180003120     ucrt:api-ms-win-crt-stdio-l1-1-0.dll
 0002:00000128       __guard_check_icall_fptr   0000000180003128     MSVCRT:guard_support.obj
 0002:00000130       __guard_xfg_check_icall_fptr 0000000180003130     MSVCRT:guard_support.obj
 0002:00000138       __guard_dispatch_icall_fptr 0000000180003138     MSVCRT:guard_support.obj
 0002:00000140       __guard_xfg_dispatch_icall_fptr 0000000180003140     MSVCRT:guard_support.obj
 0002:00000148       __guard_xfg_table_dispatch_icall_fptr 0000000180003148     MSVCRT:guard_support.obj
 0002:00000150       __castguard_check_failure_os_handled_fptr 0000000180003150     MSVCRT:guard_support.obj
 0002:00000158       __guard_memcpy_fptr        0000000180003158     vcruntime:softmemtag.obj
 0002:00000160       __xc_a                     0000000180003160     MSVCRT:initializers.obj
 0002:00000168       __xc_z                     0000000180003168     MSVCRT:initializers.obj
 0002:00000170       __xi_a                     0000000180003170     MSVCRT:initializers.obj
 0002:00000178       __xi_z                     0000000180003178     MSVCRT:initializers.obj
 0002:00000180       __xp_a                     0000000180003180     MSVCRT:initializers.obj
 0002:00000188       __xp_z                     0000000180003188     MSVCRT:initializers.obj
 0002:00000190       __xt_a                     0000000180003190     MSVCRT:initializers.obj
 0002:00000198       __xt_z                     0000000180003198     MSVCRT:initializers.obj
 0002:000001a0       ??_C@_0BI@MDECEIMI@failed?5to?5create?5thread@ 00000001800031a0     libAsyncInvokers.obj
 0002:000001b8       ??_C@_0BG@EMIOIHBI@failed?5to?5join?5thread@ 00000001800031b8     libAsyncInvokers.obj
 0002:000001d0       _pDefaultRawDllMain        00000001800031d0     MSVCRT:dll_dllmain.obj
 0002:000001d0       _pRawDllMain               00000001800031d0     MSVCRT:dll_dllmain.obj
 0002:000001f0       __xmm@ffffffffffffffffffffffffffffffff 00000001800031f0     MSVCRT:utility.obj
 0002:00000200       _load_config_used          0000000180003200     MSVCRT:loadcfg.obj
 0002:00000400       __volatile_metadata        0000000180003400     <linker-defined>
 0002:00000748       __rtc_iaa                  0000000180003748     MSVCRT:initsect.obj
 0002:00000750       __rtc_izz                  0000000180003750     MSVCRT:initsect.obj
 0002:00000758       __rtc_taa                  0000000180003758     MSVCRT:initsect.obj
 0002:00000760       __rtc_tzz                  0000000180003760     MSVCRT:initsect.obj
 0002:00001344       __IMPORT_DESCRIPTOR_KERNEL32 0000000180004344     kernel32:KERNEL32.dll
 0002:00001358       __IMPORT_DESCRIPTOR_VCRUNTIME140 0000000180004358     vcruntime:VCRUNTIME140.dll
 0002:0000136c       __IMPORT_DESCRIPTOR_api-ms-win-crt-runtime-l1-1-0 000000018000436c     ucrt:api-ms-win-crt-runtime-l1-1-0.dll
 0002:00001380       __IMPORT_DESCRIPTOR_api-ms-win-crt-stdio-l1-1-0 0000000180004380     ucrt:api-ms-win-crt-stdio-l1-1-0.dll
 0002:00001394       __NULL_IMPORT_DESCRIPTOR   0000000180004394     kernel32:KERNEL32.dll
 0003:00000000       __security_cookie          0000000180005000     MSVCRT:gs_cookie.obj
 0003:00000008       __security_cookie_complement 0000000180005008     MSVCRT:gs_cookie.obj
 0003:00000010       _fltused                   0000000180005010     MSVCRT:fltused.obj
 0003:00000014       __scrt_native_dllmain_reason 0000000180005014     MSVCRT:utility.obj
 0003:00000018       __isa_available            0000000180005018     MSVCRT:cpu_disp.obj
 0003:0000001c       __isa_enabled              000000018000501c     MSVCRT:cpu_disp.obj
 0003:00000020       __memset_fast_string_threshold 0000000180005020     MSVCRT:cpu_disp.obj
 0003:00000028       __memset_nt_threshold      0000000180005028     MSVCRT:cpu_disp.obj
 0003:00000030       __scrt_ucrt_dll_is_in_use  0000000180005030     MSVCRT:ucrt_stubs.obj
 0003:000005c0       ?__type_info_root_node@@3U__type_info_node@@A 00000001800055c0     MSVCRT:tncleanup.obj
 0003:000005d0       ?_OptionsStorage@?1??__local_stdio_printf_options@@9@4_KA 00000001800055d0     MSVCRT:default_local_stdio_options.obj
 0003:000005d8       ?_OptionsStorage@?1??__local_stdio_scanf_options@@9@4_KA 00000001800055d8     MSVCRT:default_local_stdio_options.obj
 0003:000005e0       __scrt_current_native_startup_state 00000001800055e0     MSVCRT:utility.obj
 0003:000005e8       __scrt_native_startup_lock 00000001800055e8     MSVCRT:utility.obj
 0003:00000628       __scrt_debugger_hook_flag  0000000180005628     MSVCRT:utility_desktop.obj
 0003:0000062c       __favor                    000000018000562c     MSVCRT:cpu_disp.obj
 0003:00000630       __dyn_tls_init_callback    0000000180005630     <common>

 entry point at        0001:00000d10

 Static symbols

 0000:ffff8000       .debug$S                   0000000180000000     AsyncInvokers.exp
 0000:ffff8000       .debug$S                   0000000180000000     vcruntime:VCRUNTIME140.dll
 0000:ffff8000       .debug$S                   0000000180000000     vcruntime:VCRUNTIME140.dll
 0000:ffff8000       .debug$S                   0000000180000000     vcruntime:VCRUNTIME140.dll
 0000:ffff8000       .debug$S                   0000000180000000     vcruntime:VCRUNTIME140.dll
 0000:ffff8000       .debug$S                   0000000180000000     vcruntime:VCRUNTIME140.dll
 0000:ffff8000       .debug$S                   0000000180000000     vcruntime:VCRUNTIME140.dll
 0000:ffff8000       .debug$S                   0000000180000000     ucrt:api-ms-win-crt-runtime-l1-1-0.dll
 0000:ffff8000       .debug$S                   0000000180000000     ucrt:api-ms-win-crt-runtime-l1-1-0.dll
 0000:ffff8000       .debug$S                   0000000180000000     ucrt:api-ms-win-crt-runtime-l1-1-0.dll
 0000:ffff8000       .debug$S                   0000000180000000     ucrt:api-ms-win-crt-runtime-l1-1-0.dll
 0000:ffff8000       .debug$S                   0000000180000000     ucrt:api-ms-win-crt-runtime-l1-1-0.dll
 0000:ffff8000       .debug$S                   0000000180000000     ucrt:api-ms-win-crt-runtime-l1-1-0.dll
 0000:ffff8000       .debug$S                   0000000180000000     ucrt:api-ms-win-crt-runtime-l1-1-0.dll
 0000:ffff8000       .debug$S                   0000000180000000     ucrt:api-ms-win-crt-runtime-l1-1-0.dll
 0000:ffff8000       .debug$S                   0000000180000000     ucrt:api-ms-win-crt-runtime-l1-1-0.dll
 0000:ffff8000       .debug$S                   0000000180000000     ucrt:api-ms-win-crt-runtime-l1-1-0.dll
 0000:ffff8000       .debug$S                   0000000180000000     ucrt:api-ms-win-crt-runtime-l1-1-0.dll
 0000:ffff8000       .debug$S                   0000000180000000     ucrt:api-ms-win-crt-runtime-l1-1-0.dll
 0000:ffff8000       .debug$S                   0000000180000000     ucrt:api-ms-win-crt-runtime-l1-1-0.dll
 0000:ffff8000       .debug$S                   0000000180000000     ucrt:api-ms-win-crt-stdio-l1-1-0.dll
 0000:ffff8000       .debug$S                   0000000180000000     ucrt:api-ms-win-crt-stdio-l1-1-0.dll
 0000:ffff8000       .debug$S                   0000000180000000     kernel32:KERNEL32.dll
 0000:ffff8000       .debug$S                   0000000180000000     kernel32:KERNEL32.dll
 0000:ffff8000       .debug$S                   0000000180000000     kernel32:KERNEL32.dll
 0000:ffff8000       .debug$S                   0000000180000000     kernel32:KERNEL32.dll
 0000:ffff8000       .debug$S                   0000000180000000     kernel32:KERNEL32.dll
 0000:ffff8000       .debug$S                   0000000180000000     kernel32:KERNEL32.dll
 0000:ffff8000       .debug$S                   0000000180000000     kernel32:KERNEL32.dll
 0000:ffff8000       .debug$S                   0000000180000000     kernel32:KERNEL32.dll
 0000:ffff8000       .debug$S                   0000000180000000     kernel32:KERNEL32.dll
 0000:ffff8000       .debug$S                   0000000180000000     kernel32:KERNEL32.dll
 0000:ffff8000       .debug$S                   0000000180000000     kernel32:KERNEL32.dll
 0000:ffff8000       .debug$S                   0000000180000000     kernel32:KERNEL32.dll
 0000:ffff8000       .debug$S                   0000000180000000     kernel32:KERNEL32.dll
 0000:ffff8000       .debug$S                   0000000180000000     kernel32:KERNEL32.dll
 0000:ffff8000       .debug$S                   0000000180000000     kernel32:KERNEL32.dll
 0000:ffff8000       .debug$S                   0000000180000000     kernel32:KERNEL32.dll
 0000:ffff8000       .debug$S                   0000000180000000     kernel32:KERNEL32.dll
 0000:ffff8000       .debug$S                   0000000180000000     kernel32:KERNEL32.dll
 0000:ffff8000       .debug$S                   0000000180000000     kernel32:KERNEL32.dll
 0000:ffff8000       .debug$S                   0000000180000000     kernel32:KERNEL32.dll
 0001:00000884       fatal                      0000000180001884 f   libAsyncInvokers.obj
 0001:000009c0       $$000000                   00000001800019c0     MSVCRT:amdsecgs.obj
 0001:000009f0       ?dllmain_crt_dispatch@@YAHQEAUHINSTANCE__@@KQEAX@Z 00000001800019f0 f   MSVCRT:dll_dllmain.obj
 0001:00000a40       ?dllmain_crt_process_attach@@YAHQEAUHINSTANCE__@@QEAX@Z 0000000180001a40 f   MSVCRT:dll_dllmain.obj
 0001:00000b58       ?dllmain_crt_process_detach@@YAH_N@Z 0000000180001b58 f   MSVCRT:dll_dllmain.obj
 0001:00000bdc       ?dllmain_dispatch@@YAHQEAUHINSTANCE__@@KQEAX@Z 0000000180001bdc f   MSVCRT:dll_dllmain.obj
 0001:00000e58       capture_previous_context   0000000180001e58 f   MSVCRT:gs_report.obj
 0001:00001710       $$000000                   0000000180002710     MSVCRT:guard_dispatch.obj
 0001:00001730       $$000000                   0000000180002730     MSVCRT:guard_xfg_dispatch.obj
 0001:00001746       ?fin$0@?0??dllmain_crt_process_attach@@YAHQEAUHINSTANCE__@@QEAX@Z@4HA 0000000180002746 f   MSVCRT:dll_dllmain.obj
 0001:0000175d       ?fin$0@?0??dllmain_crt_process_detach@@YAH_N@Z@4HA 000000018000275d f   MSVCRT:dll_dllmain.obj
 0001:00001776       ?fin$1@?0??dllmain_crt_process_detach@@YAH_N@Z@4HA 0000000180002776 f   MSVCRT:dll_dllmain.obj
 0001:0000178a       ?filt$0@?0??dllmain_dispatch@@YAHQEAUHINSTANCE__@@KQEAX@Z@4HA 000000018000278a f   MSVCRT:dll_dllmain.obj
 0001:000017c0       __scrt_is_nonwritable_in_current_image$filt$0 00000001800027c0 f   MSVCRT:utility.obj
 0002:000001d8       GS_ExceptionPointers       00000001800031d8     MSVCRT:gs_report.obj
 0002:00000768       $unwind$fatal              0000000180003768     libAsyncInvokers.obj
 0002:00000768       $unwind$_RTC_Initialize    0000000180003768     MSVCRT:initsect.obj
 0002:00000768       $unwind$_RTC_Terminate     0000000180003768     MSVCRT:initsect.obj
 0002:00000774       $unwind$procedure          0000000180003774     libAsyncInvokers.obj
 0002:00000774       $unwind$__scrt_initialize_default_local_stdio_options 0000000180003774     MSVCRT:default_local_stdio_options.obj
 0002:00000774       $unwind$?dllmain_crt_dispatch@@YAHQEAUHINSTANCE__@@KQEAX@Z 0000000180003774     MSVCRT:dll_dllmain.obj
 0002:00000774       $unwind$DllMain            0000000180003774     MSVCRT:dll_dllmain_stub.obj
 0002:00000774       $unwind$__GSHandlerCheck   0000000180003774     MSVCRT:gshandler.obj
 0002:00000774       $unwind$__scrt_acquire_startup_lock 0000000180003774     MSVCRT:utility.obj
 0002:00000774       $unwind$__scrt_dllmain_after_initialize_c 0000000180003774     MSVCRT:utility.obj
 0002:00000774       $unwind$__scrt_dllmain_before_initialize_c 0000000180003774     MSVCRT:utility.obj
 0002:00000774       $unwind$__scrt_dllmain_crt_thread_attach 0000000180003774     MSVCRT:utility.obj
 0002:00000774       $unwind$__scrt_dllmain_crt_thread_detach 0000000180003774     MSVCRT:utility.obj
 0002:00000774       $unwind$__scrt_dllmain_uninitialize_c 0000000180003774     MSVCRT:utility.obj
 0002:00000774       $unwind$__scrt_dllmain_uninitialize_critical 0000000180003774     MSVCRT:utility.obj
 0002:0000077c       $unwind$run_in_new_thread_and_join 000000018000377c     libAsyncInvokers.obj
 0002:00000784       $unwind$??$launch_v@P6AXXZ@@YAXP6AXXZ@Z 0000000180003784     libAsyncInvokers.obj
 0002:00000784       $unwind$??$proc_v@P6AXXZ@@YAXPEAX@Z 0000000180003784     libAsyncInvokers.obj
 0002:00000784       $unwind$call_async_D       0000000180003784     libAsyncInvokers.obj
 0002:00000784       $unwind$call_async_F       0000000180003784     libAsyncInvokers.obj
 0002:00000784       $unwind$call_async_I       0000000180003784     libAsyncInvokers.obj
 0002:00000784       $unwind$call_async_P       0000000180003784     libAsyncInvokers.obj
 0002:00000784       $unwind$call_async_V       0000000180003784     libAsyncInvokers.obj
 0002:0000078c       $unwind$??$launch@HP6AHXZ@@YAHP6AHXZ@Z 000000018000378c     libAsyncInvokers.obj
 0002:0000078c       $unwind$??$launch@MP6AMXZ@@YAMP6AMXZ@Z 000000018000378c     libAsyncInvokers.obj
 0002:0000078c       $unwind$??$launch@NP6ANXZ@@YANP6ANXZ@Z 000000018000378c     libAsyncInvokers.obj
 0002:0000078c       $unwind$??$launch@PEAXP6APEAXXZ@@YAPEAXP6APEAXXZ@Z 000000018000378c     libAsyncInvokers.obj
 0002:0000078c       $unwind$??$launch@US_D@@P6A?AU1@XZ@@YA?AUS_D@@P6A?AU0@XZ@Z 000000018000378c     libAsyncInvokers.obj
 0002:0000078c       $unwind$??$launch@US_F@@P6A?AU1@XZ@@YA?AUS_F@@P6A?AU0@XZ@Z 000000018000378c     libAsyncInvokers.obj
 0002:0000078c       $unwind$??$launch@US_FF@@P6A?AU1@XZ@@YA?AUS_FF@@P6A?AU0@XZ@Z 000000018000378c     libAsyncInvokers.obj
 0002:0000078c       $unwind$??$launch@US_FI@@P6A?AU1@XZ@@YA?AUS_FI@@P6A?AU0@XZ@Z 000000018000378c     libAsyncInvokers.obj
 0002:0000078c       $unwind$??$launch@US_I@@P6A?AU1@XZ@@YA?AUS_I@@P6A?AU0@XZ@Z 000000018000378c     libAsyncInvokers.obj
 0002:0000078c       $unwind$??$launch@US_IF@@P6A?AU1@XZ@@YA?AUS_IF@@P6A?AU0@XZ@Z 000000018000378c     libAsyncInvokers.obj
 0002:0000078c       $unwind$??$launch@US_II@@P6A?AU1@XZ@@YA?AUS_II@@P6A?AU0@XZ@Z 000000018000378c     libAsyncInvokers.obj
 0002:0000078c       $unwind$??$launch@US_P@@P6A?AU1@XZ@@YA?AUS_P@@P6A?AU0@XZ@Z 000000018000378c     libAsyncInvokers.obj
 0002:0000078c       $unwind$??$proc@HP6AHXZ@@YAXPEAX@Z 000000018000378c     libAsyncInvokers.obj
 0002:0000078c       $unwind$??$proc@MP6AMXZ@@YAXPEAX@Z 000000018000378c     libAsyncInvokers.obj
 0002:0000078c       $unwind$??$proc@NP6ANXZ@@YAXPEAX@Z 000000018000378c     libAsyncInvokers.obj
 0002:0000078c       $unwind$??$proc@PEAXP6APEAXXZ@@YAXPEAX@Z 000000018000378c     libAsyncInvokers.obj
 0002:0000078c       $unwind$??$proc@US_D@@P6A?AU1@XZ@@YAXPEAX@Z 000000018000378c     libAsyncInvokers.obj
 0002:0000078c       $unwind$??$proc@US_F@@P6A?AU1@XZ@@YAXPEAX@Z 000000018000378c     libAsyncInvokers.obj
 0002:0000078c       $unwind$??$proc@US_FF@@P6A?AU1@XZ@@YAXPEAX@Z 000000018000378c     libAsyncInvokers.obj
 0002:0000078c       $unwind$??$proc@US_FI@@P6A?AU1@XZ@@YAXPEAX@Z 000000018000378c     libAsyncInvokers.obj
 0002:0000078c       $unwind$??$proc@US_I@@P6A?AU1@XZ@@YAXPEAX@Z 000000018000378c     libAsyncInvokers.obj
 0002:0000078c       $unwind$??$proc@US_IF@@P6A?AU1@XZ@@YAXPEAX@Z 000000018000378c     libAsyncInvokers.obj
 0002:0000078c       $unwind$??$proc@US_II@@P6A?AU1@XZ@@YAXPEAX@Z 000000018000378c     libAsyncInvokers.obj
 0002:0000078c       $unwind$??$proc@US_P@@P6A?AU1@XZ@@YAXPEAX@Z 000000018000378c     libAsyncInvokers.obj
 0002:0000078c       $unwind$call_async_S_D     000000018000378c     libAsyncInvokers.obj
 0002:0000078c       $unwind$call_async_S_F     000000018000378c     libAsyncInvokers.obj
 0002:0000078c       $unwind$call_async_S_FF    000000018000378c     libAsyncInvokers.obj
 0002:0000078c       $unwind$call_async_S_FI    000000018000378c     libAsyncInvokers.obj
 0002:0000078c       $unwind$call_async_S_I     000000018000378c     libAsyncInvokers.obj
 0002:0000078c       $unwind$call_async_S_IF    000000018000378c     libAsyncInvokers.obj
 0002:0000078c       $unwind$call_async_S_II    000000018000378c     libAsyncInvokers.obj
 0002:0000078c       $unwind$call_async_S_P     000000018000378c     libAsyncInvokers.obj
 0002:0000078c       $unwind$__report_gsfailure 000000018000378c     MSVCRT:gs_report.obj
 0002:00000794       $unwind$call_async_S_DD    0000000180003794     libAsyncInvokers.obj
 0002:00000794       $unwind$call_async_S_DF    0000000180003794     libAsyncInvokers.obj
 0002:00000794       $unwind$call_async_S_DFF   0000000180003794     libAsyncInvokers.obj
 0002:00000794       $unwind$call_async_S_DFI   0000000180003794     libAsyncInvokers.obj
 0002:00000794       $unwind$call_async_S_DI    0000000180003794     libAsyncInvokers.obj
 0002:00000794       $unwind$call_async_S_DIF   0000000180003794     libAsyncInvokers.obj
 0002:00000794       $unwind$call_async_S_DII   0000000180003794     libAsyncInvokers.obj
 0002:00000794       $unwind$call_async_S_FD    0000000180003794     libAsyncInvokers.obj
 0002:00000794       $unwind$call_async_S_FFD   0000000180003794     libAsyncInvokers.obj
 0002:00000794       $unwind$call_async_S_FID   0000000180003794     libAsyncInvokers.obj
 0002:00000794       $unwind$call_async_S_ID    0000000180003794     libAsyncInvokers.obj
 0002:00000794       $unwind$call_async_S_IFD   0000000180003794     libAsyncInvokers.obj
 0002:00000794       $unwind$call_async_S_IID   0000000180003794     libAsyncInvokers.obj
 0002:000007a4       $unwind$??$launch@US_DD@@P6A?AU1@XZ@@YA?AUS_DD@@P6A?AU0@XZ@Z 00000001800037a4     libAsyncInvokers.obj
 0002:000007a4       $unwind$??$launch@US_DF@@P6A?AU1@XZ@@YA?AUS_DF@@P6A?AU0@XZ@Z 00000001800037a4     libAsyncInvokers.obj
 0002:000007a4       $unwind$??$launch@US_DFF@@P6A?AU1@XZ@@YA?AUS_DFF@@P6A?AU0@XZ@Z 00000001800037a4     libAsyncInvokers.obj
 0002:000007a4       $unwind$??$launch@US_DFI@@P6A?AU1@XZ@@YA?AUS_DFI@@P6A?AU0@XZ@Z 00000001800037a4     libAsyncInvokers.obj
 0002:000007a4       $unwind$??$launch@US_DI@@P6A?AU1@XZ@@YA?AUS_DI@@P6A?AU0@XZ@Z 00000001800037a4     libAsyncInvokers.obj
 0002:000007a4       $unwind$??$launch@US_DIF@@P6A?AU1@XZ@@YA?AUS_DIF@@P6A?AU0@XZ@Z 00000001800037a4     libAsyncInvokers.obj
 0002:000007a4       $unwind$??$launch@US_DII@@P6A?AU1@XZ@@YA?AUS_DII@@P6A?AU0@XZ@Z 00000001800037a4     libAsyncInvokers.obj
 0002:000007a4       $unwind$??$launch@US_FD@@P6A?AU1@XZ@@YA?AUS_FD@@P6A?AU0@XZ@Z 00000001800037a4     libAsyncInvokers.obj
 0002:000007a4       $unwind$??$launch@US_FFD@@P6A?AU1@XZ@@YA?AUS_FFD@@P6A?AU0@XZ@Z 00000001800037a4     libAsyncInvokers.obj
 0002:000007a4       $unwind$??$launch@US_FID@@P6A?AU1@XZ@@YA?AUS_FID@@P6A?AU0@XZ@Z 00000001800037a4     libAsyncInvokers.obj
 0002:000007a4       $unwind$??$launch@US_ID@@P6A?AU1@XZ@@YA?AUS_ID@@P6A?AU0@XZ@Z 00000001800037a4     libAsyncInvokers.obj
 0002:000007a4       $unwind$??$launch@US_IFD@@P6A?AU1@XZ@@YA?AUS_IFD@@P6A?AU0@XZ@Z 00000001800037a4     libAsyncInvokers.obj
 0002:000007a4       $unwind$??$launch@US_IID@@P6A?AU1@XZ@@YA?AUS_IID@@P6A?AU0@XZ@Z 00000001800037a4     libAsyncInvokers.obj
 0002:000007b4       $unwind$??$launch@US_DP@@P6A?AU1@XZ@@YA?AUS_DP@@P6A?AU0@XZ@Z 00000001800037b4     libAsyncInvokers.obj
 0002:000007b4       $unwind$??$launch@US_FFP@@P6A?AU1@XZ@@YA?AUS_FFP@@P6A?AU0@XZ@Z 00000001800037b4     libAsyncInvokers.obj
 0002:000007b4       $unwind$??$launch@US_FIP@@P6A?AU1@XZ@@YA?AUS_FIP@@P6A?AU0@XZ@Z 00000001800037b4     libAsyncInvokers.obj
 0002:000007b4       $unwind$??$launch@US_FP@@P6A?AU1@XZ@@YA?AUS_FP@@P6A?AU0@XZ@Z 00000001800037b4     libAsyncInvokers.obj
 0002:000007b4       $unwind$??$launch@US_IFP@@P6A?AU1@XZ@@YA?AUS_IFP@@P6A?AU0@XZ@Z 00000001800037b4     libAsyncInvokers.obj
 0002:000007b4       $unwind$??$launch@US_IIP@@P6A?AU1@XZ@@YA?AUS_IIP@@P6A?AU0@XZ@Z 00000001800037b4     libAsyncInvokers.obj
 0002:000007b4       $unwind$??$launch@US_IP@@P6A?AU1@XZ@@YA?AUS_IP@@P6A?AU0@XZ@Z 00000001800037b4     libAsyncInvokers.obj
 0002:000007b4       $unwind$??$launch@US_PD@@P6A?AU1@XZ@@YA?AUS_PD@@P6A?AU0@XZ@Z 00000001800037b4     libAsyncInvokers.obj
 0002:000007b4       $unwind$??$launch@US_PF@@P6A?AU1@XZ@@YA?AUS_PF@@P6A?AU0@XZ@Z 00000001800037b4     libAsyncInvokers.obj
 0002:000007b4       $unwind$??$launch@US_PFF@@P6A?AU1@XZ@@YA?AUS_PFF@@P6A?AU0@XZ@Z 00000001800037b4     libAsyncInvokers.obj
 0002:000007b4       $unwind$??$launch@US_PFI@@P6A?AU1@XZ@@YA?AUS_PFI@@P6A?AU0@XZ@Z 00000001800037b4     libAsyncInvokers.obj
 0002:000007b4       $unwind$??$launch@US_PI@@P6A?AU1@XZ@@YA?AUS_PI@@P6A?AU0@XZ@Z 00000001800037b4     libAsyncInvokers.obj
 0002:000007b4       $unwind$??$launch@US_PIF@@P6A?AU1@XZ@@YA?AUS_PIF@@P6A?AU0@XZ@Z 00000001800037b4     libAsyncInvokers.obj
 0002:000007b4       $unwind$??$launch@US_PII@@P6A?AU1@XZ@@YA?AUS_PII@@P6A?AU0@XZ@Z 00000001800037b4     libAsyncInvokers.obj
 0002:000007b4       $unwind$??$launch@US_PP@@P6A?AU1@XZ@@YA?AUS_PP@@P6A?AU0@XZ@Z 00000001800037b4     libAsyncInvokers.obj
 0002:000007b4       $unwind$call_async_S_DP    00000001800037b4     libAsyncInvokers.obj
 0002:000007b4       $unwind$call_async_S_FFP   00000001800037b4     libAsyncInvokers.obj
 0002:000007b4       $unwind$call_async_S_FIP   00000001800037b4     libAsyncInvokers.obj
 0002:000007b4       $unwind$call_async_S_FP    00000001800037b4     libAsyncInvokers.obj
 0002:000007b4       $unwind$call_async_S_IFP   00000001800037b4     libAsyncInvokers.obj
 0002:000007b4       $unwind$call_async_S_IIP   00000001800037b4     libAsyncInvokers.obj
 0002:000007b4       $unwind$call_async_S_IP    00000001800037b4     libAsyncInvokers.obj
 0002:000007b4       $unwind$call_async_S_PD    00000001800037b4     libAsyncInvokers.obj
 0002:000007b4       $unwind$call_async_S_PF    00000001800037b4     libAsyncInvokers.obj
 0002:000007b4       $unwind$call_async_S_PFF   00000001800037b4     libAsyncInvokers.obj
 0002:000007b4       $unwind$call_async_S_PFI   00000001800037b4     libAsyncInvokers.obj
 0002:000007b4       $unwind$call_async_S_PI    00000001800037b4     libAsyncInvokers.obj
 0002:000007b4       $unwind$call_async_S_PIF   00000001800037b4     libAsyncInvokers.obj
 0002:000007b4       $unwind$call_async_S_PII   00000001800037b4     libAsyncInvokers.obj
 0002:000007b4       $unwind$call_async_S_PP    00000001800037b4     libAsyncInvokers.obj
 0002:000007bc       $unwind$??$launch@US_DDD@@P6A?AU1@XZ@@YA?AUS_DDD@@P6A?AU0@XZ@Z 00000001800037bc     libAsyncInvokers.obj
 0002:000007bc       $unwind$??$launch@US_DDF@@P6A?AU1@XZ@@YA?AUS_DDF@@P6A?AU0@XZ@Z 00000001800037bc     libAsyncInvokers.obj
 0002:000007bc       $unwind$??$launch@US_DDI@@P6A?AU1@XZ@@YA?AUS_DDI@@P6A?AU0@XZ@Z 00000001800037bc     libAsyncInvokers.obj
 0002:000007bc       $unwind$??$launch@US_DFD@@P6A?AU1@XZ@@YA?AUS_DFD@@P6A?AU0@XZ@Z 00000001800037bc     libAsyncInvokers.obj
 0002:000007bc       $unwind$??$launch@US_DID@@P6A?AU1@XZ@@YA?AUS_DID@@P6A?AU0@XZ@Z 00000001800037bc     libAsyncInvokers.obj
 0002:000007bc       $unwind$??$launch@US_FDD@@P6A?AU1@XZ@@YA?AUS_FDD@@P6A?AU0@XZ@Z 00000001800037bc     libAsyncInvokers.obj
 0002:000007bc       $unwind$??$launch@US_FDF@@P6A?AU1@XZ@@YA?AUS_FDF@@P6A?AU0@XZ@Z 00000001800037bc     libAsyncInvokers.obj
 0002:000007bc       $unwind$??$launch@US_FDI@@P6A?AU1@XZ@@YA?AUS_FDI@@P6A?AU0@XZ@Z 00000001800037bc     libAsyncInvokers.obj
 0002:000007bc       $unwind$??$launch@US_IDD@@P6A?AU1@XZ@@YA?AUS_IDD@@P6A?AU0@XZ@Z 00000001800037bc     libAsyncInvokers.obj
 0002:000007bc       $unwind$??$launch@US_IDF@@P6A?AU1@XZ@@YA?AUS_IDF@@P6A?AU0@XZ@Z 00000001800037bc     libAsyncInvokers.obj
 0002:000007bc       $unwind$??$launch@US_IDI@@P6A?AU1@XZ@@YA?AUS_IDI@@P6A?AU0@XZ@Z 00000001800037bc     libAsyncInvokers.obj
 0002:000007bc       $unwind$call_async_S_FFF   00000001800037bc     libAsyncInvokers.obj
 0002:000007bc       $unwind$call_async_S_FFI   00000001800037bc     libAsyncInvokers.obj
 0002:000007bc       $unwind$call_async_S_FIF   00000001800037bc     libAsyncInvokers.obj
 0002:000007bc       $unwind$call_async_S_FII   00000001800037bc     libAsyncInvokers.obj
 0002:000007bc       $unwind$call_async_S_IFF   00000001800037bc     libAsyncInvokers.obj
 0002:000007bc       $unwind$call_async_S_IFI   00000001800037bc     libAsyncInvokers.obj
 0002:000007bc       $unwind$call_async_S_IIF   00000001800037bc     libAsyncInvokers.obj
 0002:000007bc       $unwind$call_async_S_III   00000001800037bc     libAsyncInvokers.obj
 0002:000007d0       $unwind$??$launch@US_FFF@@P6A?AU1@XZ@@YA?AUS_FFF@@P6A?AU0@XZ@Z 00000001800037d0     libAsyncInvokers.obj
 0002:000007d0       $unwind$??$launch@US_FFI@@P6A?AU1@XZ@@YA?AUS_FFI@@P6A?AU0@XZ@Z 00000001800037d0     libAsyncInvokers.obj
 0002:000007d0       $unwind$??$launch@US_FIF@@P6A?AU1@XZ@@YA?AUS_FIF@@P6A?AU0@XZ@Z 00000001800037d0     libAsyncInvokers.obj
 0002:000007d0       $unwind$??$launch@US_FII@@P6A?AU1@XZ@@YA?AUS_FII@@P6A?AU0@XZ@Z 00000001800037d0     libAsyncInvokers.obj
 0002:000007d0       $unwind$??$launch@US_IFF@@P6A?AU1@XZ@@YA?AUS_IFF@@P6A?AU0@XZ@Z 00000001800037d0     libAsyncInvokers.obj
 0002:000007d0       $unwind$??$launch@US_IFI@@P6A?AU1@XZ@@YA?AUS_IFI@@P6A?AU0@XZ@Z 00000001800037d0     libAsyncInvokers.obj
 0002:000007d0       $unwind$??$launch@US_IIF@@P6A?AU1@XZ@@YA?AUS_IIF@@P6A?AU0@XZ@Z 00000001800037d0     libAsyncInvokers.obj
 0002:000007d0       $unwind$??$launch@US_III@@P6A?AU1@XZ@@YA?AUS_III@@P6A?AU0@XZ@Z 00000001800037d0     libAsyncInvokers.obj
 0002:000007e4       $unwind$call_async_S_DDD   00000001800037e4     libAsyncInvokers.obj
 0002:000007e4       $unwind$call_async_S_DDF   00000001800037e4     libAsyncInvokers.obj
 0002:000007e4       $unwind$call_async_S_DDI   00000001800037e4     libAsyncInvokers.obj
 0002:000007e4       $unwind$call_async_S_DFD   00000001800037e4     libAsyncInvokers.obj
 0002:000007e4       $unwind$call_async_S_DID   00000001800037e4     libAsyncInvokers.obj
 0002:000007e4       $unwind$call_async_S_FDD   00000001800037e4     libAsyncInvokers.obj
 0002:000007e4       $unwind$call_async_S_FDF   00000001800037e4     libAsyncInvokers.obj
 0002:000007e4       $unwind$call_async_S_FDI   00000001800037e4     libAsyncInvokers.obj
 0002:000007e4       $unwind$call_async_S_IDD   00000001800037e4     libAsyncInvokers.obj
 0002:000007e4       $unwind$call_async_S_IDF   00000001800037e4     libAsyncInvokers.obj
 0002:000007e4       $unwind$call_async_S_IDI   00000001800037e4     libAsyncInvokers.obj
 0002:000007f8       $unwind$call_async_S_DDP   00000001800037f8     libAsyncInvokers.obj
 0002:000007f8       $unwind$call_async_S_DFP   00000001800037f8     libAsyncInvokers.obj
 0002:000007f8       $unwind$call_async_S_DIP   00000001800037f8     libAsyncInvokers.obj
 0002:000007f8       $unwind$call_async_S_DPD   00000001800037f8     libAsyncInvokers.obj
 0002:000007f8       $unwind$call_async_S_DPF   00000001800037f8     libAsyncInvokers.obj
 0002:000007f8       $unwind$call_async_S_DPI   00000001800037f8     libAsyncInvokers.obj
 0002:000007f8       $unwind$call_async_S_DPP   00000001800037f8     libAsyncInvokers.obj
 0002:000007f8       $unwind$call_async_S_FDP   00000001800037f8     libAsyncInvokers.obj
 0002:000007f8       $unwind$call_async_S_FPD   00000001800037f8     libAsyncInvokers.obj
 0002:000007f8       $unwind$call_async_S_FPF   00000001800037f8     libAsyncInvokers.obj
 0002:000007f8       $unwind$call_async_S_FPI   00000001800037f8     libAsyncInvokers.obj
 0002:000007f8       $unwind$call_async_S_FPP   00000001800037f8     libAsyncInvokers.obj
 0002:000007f8       $unwind$call_async_S_IDP   00000001800037f8     libAsyncInvokers.obj
 0002:000007f8       $unwind$call_async_S_IPD   00000001800037f8     libAsyncInvokers.obj
 0002:000007f8       $unwind$call_async_S_IPF   00000001800037f8     libAsyncInvokers.obj
 0002:000007f8       $unwind$call_async_S_IPI   00000001800037f8     libAsyncInvokers.obj
 0002:000007f8       $unwind$call_async_S_IPP   00000001800037f8     libAsyncInvokers.obj
 0002:000007f8       $unwind$call_async_S_PDD   00000001800037f8     libAsyncInvokers.obj
 0002:000007f8       $unwind$call_async_S_PDF   00000001800037f8     libAsyncInvokers.obj
 0002:000007f8       $unwind$call_async_S_PDI   00000001800037f8     libAsyncInvokers.obj
 0002:000007f8       $unwind$call_async_S_PDP   00000001800037f8     libAsyncInvokers.obj
 0002:000007f8       $unwind$call_async_S_PFD   00000001800037f8     libAsyncInvokers.obj
 0002:000007f8       $unwind$call_async_S_PFP   00000001800037f8     libAsyncInvokers.obj
 0002:000007f8       $unwind$call_async_S_PID   00000001800037f8     libAsyncInvokers.obj
 0002:000007f8       $unwind$call_async_S_PIP   00000001800037f8     libAsyncInvokers.obj
 0002:000007f8       $unwind$call_async_S_PPD   00000001800037f8     libAsyncInvokers.obj
 0002:000007f8       $unwind$call_async_S_PPF   00000001800037f8     libAsyncInvokers.obj
 0002:000007f8       $unwind$call_async_S_PPI   00000001800037f8     libAsyncInvokers.obj
 0002:000007f8       $unwind$call_async_S_PPP   00000001800037f8     libAsyncInvokers.obj
 0002:00000804       $unwind$??$launch@US_DDP@@P6A?AU1@XZ@@YA?AUS_DDP@@P6A?AU0@XZ@Z 0000000180003804     libAsyncInvokers.obj
 0002:00000804       $unwind$??$launch@US_DFP@@P6A?AU1@XZ@@YA?AUS_DFP@@P6A?AU0@XZ@Z 0000000180003804     libAsyncInvokers.obj
 0002:00000804       $unwind$??$launch@US_DIP@@P6A?AU1@XZ@@YA?AUS_DIP@@P6A?AU0@XZ@Z 0000000180003804     libAsyncInvokers.obj
 0002:00000804       $unwind$??$launch@US_DPD@@P6A?AU1@XZ@@YA?AUS_DPD@@P6A?AU0@XZ@Z 0000000180003804     libAsyncInvokers.obj
 0002:00000804       $unwind$??$launch@US_DPF@@P6A?AU1@XZ@@YA?AUS_DPF@@P6A?AU0@XZ@Z 0000000180003804     libAsyncInvokers.obj
 0002:00000804       $unwind$??$launch@US_DPI@@P6A?AU1@XZ@@YA?AUS_DPI@@P6A?AU0@XZ@Z 0000000180003804     libAsyncInvokers.obj
 0002:00000804       $unwind$??$launch@US_DPP@@P6A?AU1@XZ@@YA?AUS_DPP@@P6A?AU0@XZ@Z 0000000180003804     libAsyncInvokers.obj
 0002:00000804       $unwind$??$launch@US_FDP@@P6A?AU1@XZ@@YA?AUS_FDP@@P6A?AU0@XZ@Z 0000000180003804     libAsyncInvokers.obj
 0002:00000804       $unwind$??$launch@US_FPD@@P6A?AU1@XZ@@YA?AUS_FPD@@P6A?AU0@XZ@Z 0000000180003804     libAsyncInvokers.obj
 0002:00000804       $unwind$??$launch@US_FPF@@P6A?AU1@XZ@@YA?AUS_FPF@@P6A?AU0@XZ@Z 0000000180003804     libAsyncInvokers.obj
 0002:00000804       $unwind$??$launch@US_FPI@@P6A?AU1@XZ@@YA?AUS_FPI@@P6A?AU0@XZ@Z 0000000180003804     libAsyncInvokers.obj
 0002:00000804       $unwind$??$launch@US_FPP@@P6A?AU1@XZ@@YA?AUS_FPP@@P6A?AU0@XZ@Z 0000000180003804     libAsyncInvokers.obj
 0002:00000804       $unwind$??$launch@US_IDP@@P6A?AU1@XZ@@YA?AUS_IDP@@P6A?AU0@XZ@Z 0000000180003804     libAsyncInvokers.obj
 0002:00000804       $unwind$??$launch@US_IPD@@P6A?AU1@XZ@@YA?AUS_IPD@@P6A?AU0@XZ@Z 0000000180003804     libAsyncInvokers.obj
 0002:00000804       $unwind$??$launch@US_IPF@@P6A?AU1@XZ@@YA?AUS_IPF@@P6A?AU0@XZ@Z 0000000180003804     libAsyncInvokers.obj
 0002:00000804       $unwind$??$launch@US_IPI@@P6A?AU1@XZ@@YA?AUS_IPI@@P6A?AU0@XZ@Z 0000000180003804     libAsyncInvokers.obj
 0002:00000804       $unwind$??$launch@US_IPP@@P6A?AU1@XZ@@YA?AUS_IPP@@P6A?AU0@XZ@Z 0000000180003804     libAsyncInvokers.obj
 0002:00000804       $unwind$??$launch@US_PDD@@P6A?AU1@XZ@@YA?AUS_PDD@@P6A?AU0@XZ@Z 0000000180003804     libAsyncInvokers.obj
 0002:00000804       $unwind$??$launch@US_PDF@@P6A?AU1@XZ@@YA?AUS_PDF@@P6A?AU0@XZ@Z 0000000180003804     libAsyncInvokers.obj
 0002:00000804       $unwind$??$launch@US_PDI@@P6A?AU1@XZ@@YA?AUS_PDI@@P6A?AU0@XZ@Z 0000000180003804     libAsyncInvokers.obj
 0002:00000804       $unwind$??$launch@US_PDP@@P6A?AU1@XZ@@YA?AUS_PDP@@P6A?AU0@XZ@Z 0000000180003804     libAsyncInvokers.obj
 0002:00000804       $unwind$??$launch@US_PFD@@P6A?AU1@XZ@@YA?AUS_PFD@@P6A?AU0@XZ@Z 0000000180003804     libAsyncInvokers.obj
 0002:00000804       $unwind$??$launch@US_PFP@@P6A?AU1@XZ@@YA?AUS_PFP@@P6A?AU0@XZ@Z 0000000180003804     libAsyncInvokers.obj
 0002:00000804       $unwind$??$launch@US_PID@@P6A?AU1@XZ@@YA?AUS_PID@@P6A?AU0@XZ@Z 0000000180003804     libAsyncInvokers.obj
 0002:00000804       $unwind$??$launch@US_PIP@@P6A?AU1@XZ@@YA?AUS_PIP@@P6A?AU0@XZ@Z 0000000180003804     libAsyncInvokers.obj
 0002:00000804       $unwind$??$launch@US_PPD@@P6A?AU1@XZ@@YA?AUS_PPD@@P6A?AU0@XZ@Z 0000000180003804     libAsyncInvokers.obj
 0002:00000804       $unwind$??$launch@US_PPF@@P6A?AU1@XZ@@YA?AUS_PPF@@P6A?AU0@XZ@Z 0000000180003804     libAsyncInvokers.obj
 0002:00000804       $unwind$??$launch@US_PPI@@P6A?AU1@XZ@@YA?AUS_PPI@@P6A?AU0@XZ@Z 0000000180003804     libAsyncInvokers.obj
 0002:00000804       $unwind$??$launch@US_PPP@@P6A?AU1@XZ@@YA?AUS_PPP@@P6A?AU0@XZ@Z 0000000180003804     libAsyncInvokers.obj
 0002:00000810       $unwind$??$proc@US_DD@@P6A?AU1@XZ@@YAXPEAX@Z 0000000180003810     libAsyncInvokers.obj
 0002:00000810       $unwind$??$proc@US_DF@@P6A?AU1@XZ@@YAXPEAX@Z 0000000180003810     libAsyncInvokers.obj
 0002:00000810       $unwind$??$proc@US_DFF@@P6A?AU1@XZ@@YAXPEAX@Z 0000000180003810     libAsyncInvokers.obj
 0002:00000810       $unwind$??$proc@US_DFI@@P6A?AU1@XZ@@YAXPEAX@Z 0000000180003810     libAsyncInvokers.obj
 0002:00000810       $unwind$??$proc@US_DI@@P6A?AU1@XZ@@YAXPEAX@Z 0000000180003810     libAsyncInvokers.obj
 0002:00000810       $unwind$??$proc@US_DIF@@P6A?AU1@XZ@@YAXPEAX@Z 0000000180003810     libAsyncInvokers.obj
 0002:00000810       $unwind$??$proc@US_DII@@P6A?AU1@XZ@@YAXPEAX@Z 0000000180003810     libAsyncInvokers.obj
 0002:00000810       $unwind$??$proc@US_FD@@P6A?AU1@XZ@@YAXPEAX@Z 0000000180003810     libAsyncInvokers.obj
 0002:00000810       $unwind$??$proc@US_FFD@@P6A?AU1@XZ@@YAXPEAX@Z 0000000180003810     libAsyncInvokers.obj
 0002:00000810       $unwind$??$proc@US_FID@@P6A?AU1@XZ@@YAXPEAX@Z 0000000180003810     libAsyncInvokers.obj
 0002:00000810       $unwind$??$proc@US_ID@@P6A?AU1@XZ@@YAXPEAX@Z 0000000180003810     libAsyncInvokers.obj
 0002:00000810       $unwind$??$proc@US_IFD@@P6A?AU1@XZ@@YAXPEAX@Z 0000000180003810     libAsyncInvokers.obj
 0002:00000810       $unwind$??$proc@US_IID@@P6A?AU1@XZ@@YAXPEAX@Z 0000000180003810     libAsyncInvokers.obj
 0002:00000820       $unwind$??$proc@US_DP@@P6A?AU1@XZ@@YAXPEAX@Z 0000000180003820     libAsyncInvokers.obj
 0002:00000820       $unwind$??$proc@US_FFP@@P6A?AU1@XZ@@YAXPEAX@Z 0000000180003820     libAsyncInvokers.obj
 0002:00000820       $unwind$??$proc@US_FIP@@P6A?AU1@XZ@@YAXPEAX@Z 0000000180003820     libAsyncInvokers.obj
 0002:00000820       $unwind$??$proc@US_FP@@P6A?AU1@XZ@@YAXPEAX@Z 0000000180003820     libAsyncInvokers.obj
 0002:00000820       $unwind$??$proc@US_IFP@@P6A?AU1@XZ@@YAXPEAX@Z 0000000180003820     libAsyncInvokers.obj
 0002:00000820       $unwind$??$proc@US_IIP@@P6A?AU1@XZ@@YAXPEAX@Z 0000000180003820     libAsyncInvokers.obj
 0002:00000820       $unwind$??$proc@US_IP@@P6A?AU1@XZ@@YAXPEAX@Z 0000000180003820     libAsyncInvokers.obj
 0002:00000820       $unwind$??$proc@US_PD@@P6A?AU1@XZ@@YAXPEAX@Z 0000000180003820     libAsyncInvokers.obj
 0002:00000820       $unwind$??$proc@US_PF@@P6A?AU1@XZ@@YAXPEAX@Z 0000000180003820     libAsyncInvokers.obj
 0002:00000820       $unwind$??$proc@US_PFF@@P6A?AU1@XZ@@YAXPEAX@Z 0000000180003820     libAsyncInvokers.obj
 0002:00000820       $unwind$??$proc@US_PFI@@P6A?AU1@XZ@@YAXPEAX@Z 0000000180003820     libAsyncInvokers.obj
 0002:00000820       $unwind$??$proc@US_PI@@P6A?AU1@XZ@@YAXPEAX@Z 0000000180003820     libAsyncInvokers.obj
 0002:00000820       $unwind$??$proc@US_PIF@@P6A?AU1@XZ@@YAXPEAX@Z 0000000180003820     libAsyncInvokers.obj
 0002:00000820       $unwind$??$proc@US_PII@@P6A?AU1@XZ@@YAXPEAX@Z 0000000180003820     libAsyncInvokers.obj
 0002:00000820       $unwind$??$proc@US_PP@@P6A?AU1@XZ@@YAXPEAX@Z 0000000180003820     libAsyncInvokers.obj
 0002:00000828       $unwind$??$proc@US_FFF@@P6A?AU1@XZ@@YAXPEAX@Z 0000000180003828     libAsyncInvokers.obj
 0002:00000828       $unwind$??$proc@US_FFI@@P6A?AU1@XZ@@YAXPEAX@Z 0000000180003828     libAsyncInvokers.obj
 0002:00000828       $unwind$??$proc@US_FIF@@P6A?AU1@XZ@@YAXPEAX@Z 0000000180003828     libAsyncInvokers.obj
 0002:00000828       $unwind$??$proc@US_FII@@P6A?AU1@XZ@@YAXPEAX@Z 0000000180003828     libAsyncInvokers.obj
 0002:00000828       $unwind$??$proc@US_IFF@@P6A?AU1@XZ@@YAXPEAX@Z 0000000180003828     libAsyncInvokers.obj
 0002:00000828       $unwind$??$proc@US_IFI@@P6A?AU1@XZ@@YAXPEAX@Z 0000000180003828     libAsyncInvokers.obj
 0002:00000828       $unwind$??$proc@US_IIF@@P6A?AU1@XZ@@YAXPEAX@Z 0000000180003828     libAsyncInvokers.obj
 0002:00000828       $unwind$??$proc@US_III@@P6A?AU1@XZ@@YAXPEAX@Z 0000000180003828     libAsyncInvokers.obj
 0002:0000083c       $unwind$??$proc@US_DDD@@P6A?AU1@XZ@@YAXPEAX@Z 000000018000383c     libAsyncInvokers.obj
 0002:0000083c       $unwind$??$proc@US_DDF@@P6A?AU1@XZ@@YAXPEAX@Z 000000018000383c     libAsyncInvokers.obj
 0002:0000083c       $unwind$??$proc@US_DDI@@P6A?AU1@XZ@@YAXPEAX@Z 000000018000383c     libAsyncInvokers.obj
 0002:0000083c       $unwind$??$proc@US_DFD@@P6A?AU1@XZ@@YAXPEAX@Z 000000018000383c     libAsyncInvokers.obj
 0002:0000083c       $unwind$??$proc@US_DID@@P6A?AU1@XZ@@YAXPEAX@Z 000000018000383c     libAsyncInvokers.obj
 0002:0000083c       $unwind$??$proc@US_FDD@@P6A?AU1@XZ@@YAXPEAX@Z 000000018000383c     libAsyncInvokers.obj
 0002:0000083c       $unwind$??$proc@US_FDF@@P6A?AU1@XZ@@YAXPEAX@Z 000000018000383c     libAsyncInvokers.obj
 0002:0000083c       $unwind$??$proc@US_FDI@@P6A?AU1@XZ@@YAXPEAX@Z 000000018000383c     libAsyncInvokers.obj
 0002:0000083c       $unwind$??$proc@US_IDD@@P6A?AU1@XZ@@YAXPEAX@Z 000000018000383c     libAsyncInvokers.obj
 0002:0000083c       $unwind$??$proc@US_IDF@@P6A?AU1@XZ@@YAXPEAX@Z 000000018000383c     libAsyncInvokers.obj
 0002:0000083c       $unwind$??$proc@US_IDI@@P6A?AU1@XZ@@YAXPEAX@Z 000000018000383c     libAsyncInvokers.obj
 0002:00000850       $unwind$??$proc@US_DDP@@P6A?AU1@XZ@@YAXPEAX@Z 0000000180003850     libAsyncInvokers.obj
 0002:00000850       $unwind$??$proc@US_DFP@@P6A?AU1@XZ@@YAXPEAX@Z 0000000180003850     libAsyncInvokers.obj
 0002:00000850       $unwind$??$proc@US_DIP@@P6A?AU1@XZ@@YAXPEAX@Z 0000000180003850     libAsyncInvokers.obj
 0002:00000850       $unwind$??$proc@US_DPD@@P6A?AU1@XZ@@YAXPEAX@Z 0000000180003850     libAsyncInvokers.obj
 0002:00000850       $unwind$??$proc@US_DPF@@P6A?AU1@XZ@@YAXPEAX@Z 0000000180003850     libAsyncInvokers.obj
 0002:00000850       $unwind$??$proc@US_DPI@@P6A?AU1@XZ@@YAXPEAX@Z 0000000180003850     libAsyncInvokers.obj
 0002:00000850       $unwind$??$proc@US_DPP@@P6A?AU1@XZ@@YAXPEAX@Z 0000000180003850     libAsyncInvokers.obj
 0002:00000850       $unwind$??$proc@US_FDP@@P6A?AU1@XZ@@YAXPEAX@Z 0000000180003850     libAsyncInvokers.obj
 0002:00000850       $unwind$??$proc@US_FPD@@P6A?AU1@XZ@@YAXPEAX@Z 0000000180003850     libAsyncInvokers.obj
 0002:00000850       $unwind$??$proc@US_FPF@@P6A?AU1@XZ@@YAXPEAX@Z 0000000180003850     libAsyncInvokers.obj
 0002:00000850       $unwind$??$proc@US_FPI@@P6A?AU1@XZ@@YAXPEAX@Z 0000000180003850     libAsyncInvokers.obj
 0002:00000850       $unwind$??$proc@US_FPP@@P6A?AU1@XZ@@YAXPEAX@Z 0000000180003850     libAsyncInvokers.obj
 0002:00000850       $unwind$??$proc@US_IDP@@P6A?AU1@XZ@@YAXPEAX@Z 0000000180003850     libAsyncInvokers.obj
 0002:00000850       $unwind$??$proc@US_IPD@@P6A?AU1@XZ@@YAXPEAX@Z 0000000180003850     libAsyncInvokers.obj
 0002:00000850       $unwind$??$proc@US_IPF@@P6A?AU1@XZ@@YAXPEAX@Z 0000000180003850     libAsyncInvokers.obj
 0002:00000850       $unwind$??$proc@US_IPI@@P6A?AU1@XZ@@YAXPEAX@Z 0000000180003850     libAsyncInvokers.obj
 0002:00000850       $unwind$??$proc@US_IPP@@P6A?AU1@XZ@@YAXPEAX@Z 0000000180003850     libAsyncInvokers.obj
 0002:00000850       $unwind$??$proc@US_PDD@@P6A?AU1@XZ@@YAXPEAX@Z 0000000180003850     libAsyncInvokers.obj
 0002:00000850       $unwind$??$proc@US_PDF@@P6A?AU1@XZ@@YAXPEAX@Z 0000000180003850     libAsyncInvokers.obj
 0002:00000850       $unwind$??$proc@US_PDI@@P6A?AU1@XZ@@YAXPEAX@Z 0000000180003850     libAsyncInvokers.obj
 0002:00000850       $unwind$??$proc@US_PDP@@P6A?AU1@XZ@@YAXPEAX@Z 0000000180003850     libAsyncInvokers.obj
 0002:00000850       $unwind$??$proc@US_PFD@@P6A?AU1@XZ@@YAXPEAX@Z 0000000180003850     libAsyncInvokers.obj
 0002:00000850       $unwind$??$proc@US_PFP@@P6A?AU1@XZ@@YAXPEAX@Z 0000000180003850     libAsyncInvokers.obj
 0002:00000850       $unwind$??$proc@US_PID@@P6A?AU1@XZ@@YAXPEAX@Z 0000000180003850     libAsyncInvokers.obj
 0002:00000850       $unwind$??$proc@US_PIP@@P6A?AU1@XZ@@YAXPEAX@Z 0000000180003850     libAsyncInvokers.obj
 0002:00000850       $unwind$??$proc@US_PPD@@P6A?AU1@XZ@@YAXPEAX@Z 0000000180003850     libAsyncInvokers.obj
 0002:00000850       $unwind$??$proc@US_PPF@@P6A?AU1@XZ@@YAXPEAX@Z 0000000180003850     libAsyncInvokers.obj
 0002:00000850       $unwind$??$proc@US_PPI@@P6A?AU1@XZ@@YAXPEAX@Z 0000000180003850     libAsyncInvokers.obj
 0002:00000850       $unwind$??$proc@US_PPP@@P6A?AU1@XZ@@YAXPEAX@Z 0000000180003850     libAsyncInvokers.obj
 0002:0000085c       $unwind$__GSHandlerCheckCommon 000000018000385c     MSVCRT:gshandler.obj
 0002:00000868       $xdatasym                  0000000180003868     MSVCRT:amdsecgs.obj
 0002:0000086c       $unwind$?dllmain_crt_process_attach@@YAHQEAUHINSTANCE__@@QEAX@Z 000000018000386c     MSVCRT:dll_dllmain.obj
 0002:000008a8       $unwind$?fin$0@?0??dllmain_crt_process_attach@@YAHQEAUHINSTANCE__@@QEAX@Z@4HA 00000001800038a8     MSVCRT:dll_dllmain.obj
 0002:000008a8       $unwind$?fin$0@?0??dllmain_crt_process_detach@@YAH_N@Z@4HA 00000001800038a8     MSVCRT:dll_dllmain.obj
 0002:000008a8       $unwind$?fin$1@?0??dllmain_crt_process_detach@@YAH_N@Z@4HA 00000001800038a8     MSVCRT:dll_dllmain.obj
 0002:000008b0       $unwind$?dllmain_crt_process_detach@@YAH_N@Z 00000001800038b0     MSVCRT:dll_dllmain.obj
 0002:00000904       $unwind$?dllmain_dispatch@@YAHQEAUHINSTANCE__@@KQEAX@Z 0000000180003904     MSVCRT:dll_dllmain.obj
 0002:0000092c       $unwind$?filt$0@?0??dllmain_dispatch@@YAHQEAUHINSTANCE__@@KQEAX@Z@4HA 000000018000392c     MSVCRT:dll_dllmain.obj
 0002:00000934       $unwind$_DllMainCRTStartup 0000000180003934     MSVCRT:dll_dllmain.obj
 0002:00000944       $unwind$capture_previous_context 0000000180003944     MSVCRT:gs_report.obj
 0002:00000950       $unwind$__raise_securityfailure 0000000180003950     MSVCRT:gs_report.obj
 0002:00000950       $unwind$__scrt_initialize_crt 0000000180003950     MSVCRT:utility.obj
 0002:00000950       $unwind$__scrt_initialize_onexit_tables 0000000180003950     MSVCRT:utility.obj
 0002:00000950       $unwind$__scrt_release_startup_lock 0000000180003950     MSVCRT:utility.obj
 0002:00000950       $unwind$__scrt_uninitialize_crt 0000000180003950     MSVCRT:utility.obj
 0002:00000958       $unwind$__security_init_cookie 0000000180003958     MSVCRT:gs_support.obj
 0002:00000964       $unwind$__scrt_is_nonwritable_in_current_image 0000000180003964     MSVCRT:utility.obj
 0002:00000984       $unwind$__scrt_is_nonwritable_in_current_image$filt$0 0000000180003984     MSVCRT:utility.obj
 0002:0000098c       $unwind$__scrt_dllmain_exception_filter 000000018000398c     MSVCRT:utility.obj
 0002:000009a0       $unwind$__scrt_fastfail    00000001800039a0     MSVCRT:utility_desktop.obj
 0002:000009b0       $unwind$__isa_available_init 00000001800039b0     MSVCRT:cpu_disp.obj
 0002:000009c0       $xdatasym                  00000001800039c0     MSVCRT:guard_dispatch.obj
 0002:000009c8       $xdatasym                  00000001800039c8     MSVCRT:guard_xfg_dispatch.obj
 0002:000009d0       .edata                     00000001800039d0     AsyncInvokers.exp
 0002:000009f8       rgpv                       00000001800039f8     AsyncInvokers.exp
 0002:00000b5c       rgszName                   0000000180003b5c     AsyncInvokers.exp
 0002:00000cc0       rgwOrd                     0000000180003cc0     AsyncInvokers.exp
 0002:00000d72       szName                     0000000180003d72     AsyncInvokers.exp
 0002:00000d84       $N00001                    0000000180003d84     AsyncInvokers.exp
 0002:00000d91       $N00002                    0000000180003d91     AsyncInvokers.exp
 0002:00000d9e       $N00003                    0000000180003d9e     AsyncInvokers.exp
 0002:00000dab       $N00004                    0000000180003dab     AsyncInvokers.exp
 0002:00000db8       $N00005                    0000000180003db8     AsyncInvokers.exp
 0002:00000dc7       $N00006                    0000000180003dc7     AsyncInvokers.exp
 0002:00000dd7       $N00007                    0000000180003dd7     AsyncInvokers.exp
 0002:00000de8       $N00008                    0000000180003de8     AsyncInvokers.exp
 0002:00000df9       $N00009                    0000000180003df9     AsyncInvokers.exp
 0002:00000e0a       $N00010                    0000000180003e0a     AsyncInvokers.exp
 0002:00000e1b       $N00011                    0000000180003e1b     AsyncInvokers.exp
 0002:00000e2b       $N00012                    0000000180003e2b     AsyncInvokers.exp
 0002:00000e3c       $N00013                    0000000180003e3c     AsyncInvokers.exp
 0002:00000e4d       $N00014                    0000000180003e4d     AsyncInvokers.exp
 0002:00000e5e       $N00015                    0000000180003e5e     AsyncInvokers.exp
 0002:00000e6f       $N00016                    0000000180003e6f     AsyncInvokers.exp
 0002:00000e7f       $N00017                    0000000180003e7f     AsyncInvokers.exp
 0002:00000e90       $N00018                    0000000180003e90     AsyncInvokers.exp
 0002:00000ea1       $N00019                    0000000180003ea1     AsyncInvokers.exp
 0002:00000eb2       $N00020                    0000000180003eb2     AsyncInvokers.exp
 0002:00000ec3       $N00021                    0000000180003ec3     AsyncInvokers.exp
 0002:00000ed3       $N00022                    0000000180003ed3     AsyncInvokers.exp
 0002:00000ee4       $N00023                    0000000180003ee4     AsyncInvokers.exp
 0002:00000ef5       $N00024                    0000000180003ef5     AsyncInvokers.exp
 0002:00000f06       $N00025                    0000000180003f06     AsyncInvokers.exp
 0002:00000f17       $N00026                    0000000180003f17     AsyncInvokers.exp
 0002:00000f26       $N00027                    0000000180003f26     AsyncInvokers.exp
 0002:00000f36       $N00028                    0000000180003f36     AsyncInvokers.exp
 0002:00000f47       $N00029                    0000000180003f47     AsyncInvokers.exp
 0002:00000f58       $N00030                    0000000180003f58     AsyncInvokers.exp
 0002:00000f69       $N00031                    0000000180003f69     AsyncInvokers.exp
 0002:00000f7a       $N00032                    0000000180003f7a     AsyncInvokers.exp
 0002:00000f8a       $N00033                    0000000180003f8a     AsyncInvokers.exp
 0002:00000f9b       $N00034                    0000000180003f9b     AsyncInvokers.exp
 0002:00000fac       $N00035                    0000000180003fac     AsyncInvokers.exp
 0002:00000fbd       $N00036                    0000000180003fbd     AsyncInvokers.exp
 0002:00000fce       $N00037                    0000000180003fce     AsyncInvokers.exp
 0002:00000fde       $N00038                    0000000180003fde     AsyncInvokers.exp
 0002:00000fef       $N00039                    0000000180003fef     AsyncInvokers.exp
 0002:00001000       $N00040                    0000000180004000     AsyncInvokers.exp
 0002:00001011       $N00041                    0000000180004011     AsyncInvokers.exp
 0002:00001022       $N00042                    0000000180004022     AsyncInvokers.exp
 0002:00001032       $N00043                    0000000180004032     AsyncInvokers.exp
 0002:00001043       $N00044                    0000000180004043     AsyncInvokers.exp
 0002:00001054       $N00045                    0000000180004054     AsyncInvokers.exp
 0002:00001065       $N00046                    0000000180004065     AsyncInvokers.exp
 0002:00001076       $N00047                    0000000180004076     AsyncInvokers.exp
 0002:00001085       $N00048                    0000000180004085     AsyncInvokers.exp
 0002:00001095       $N00049                    0000000180004095     AsyncInvokers.exp
 0002:000010a6       $N00050                    00000001800040a6     AsyncInvokers.exp
 0002:000010b7       $N00051                    00000001800040b7     AsyncInvokers.exp
 0002:000010c8       $N00052                    00000001800040c8     AsyncInvokers.exp
 0002:000010d9       $N00053                    00000001800040d9     AsyncInvokers.exp
 0002:000010e9       $N00054                    00000001800040e9     AsyncInvokers.exp
 0002:000010fa       $N00055                    00000001800040fa     AsyncInvokers.exp
 0002:0000110b       $N00056                    000000018000410b     AsyncInvokers.exp
 0002:0000111c       $N00057                    000000018000411c     AsyncInvokers.exp
 0002:0000112d       $N00058                    000000018000412d     AsyncInvokers.exp
 0002:0000113d       $N00059                    000000018000413d     AsyncInvokers.exp
 0002:0000114e       $N00060                    000000018000414e     AsyncInvokers.exp
 0002:0000115f       $N00061                    000000018000415f     AsyncInvokers.exp
 0002:00001170       $N00062                    0000000180004170     AsyncInvokers.exp
 0002:00001181       $N00063                    0000000180004181     AsyncInvokers.exp
 0002:00001191       $N00064                    0000000180004191     AsyncInvokers.exp
 0002:000011a2       $N00065                    00000001800041a2     AsyncInvokers.exp
 0002:000011b3       $N00066                    00000001800041b3     AsyncInvokers.exp
 0002:000011c4       $N00067                    00000001800041c4     AsyncInvokers.exp
 0002:000011d5       $N00068                    00000001800041d5     AsyncInvokers.exp
 0002:000011e4       $N00069                    00000001800041e4     AsyncInvokers.exp
 0002:000011f4       $N00070                    00000001800041f4     AsyncInvokers.exp
 0002:00001205       $N00071                    0000000180004205     AsyncInvokers.exp
 0002:00001216       $N00072                    0000000180004216     AsyncInvokers.exp
 0002:00001227       $N00073                    0000000180004227     AsyncInvokers.exp
 0002:00001238       $N00074                    0000000180004238     AsyncInvokers.exp
 0002:00001248       $N00075                    0000000180004248     AsyncInvokers.exp
 0002:00001259       $N00076                    0000000180004259     AsyncInvokers.exp
 0002:0000126a       $N00077                    000000018000426a     AsyncInvokers.exp
 0002:0000127b       $N00078                    000000018000427b     AsyncInvokers.exp
 0002:0000128c       $N00079                    000000018000428c     AsyncInvokers.exp
 0002:0000129c       $N00080                    000000018000429c     AsyncInvokers.exp
 0002:000012ad       $N00081                    00000001800042ad     AsyncInvokers.exp
 0002:000012be       $N00082                    00000001800042be     AsyncInvokers.exp
 0002:000012cf       $N00083                    00000001800042cf     AsyncInvokers.exp
 0002:000012e0       $N00084                    00000001800042e0     AsyncInvokers.exp
 0002:000012f0       $N00085                    00000001800042f0     AsyncInvokers.exp
 0002:00001301       $N00086                    0000000180004301     AsyncInvokers.exp
 0002:00001312       $N00087                    0000000180004312     AsyncInvokers.exp
 0002:00001323       $N00088                    0000000180004323     AsyncInvokers.exp
 0002:00001334       $N00089                    0000000180004334     AsyncInvokers.exp
 0002:0000166c       .idata$6                   000000018000466c     kernel32:KERNEL32.dll
 0002:000016bc       .idata$6                   00000001800046bc     vcruntime:VCRUNTIME140.dll
 0002:00001796       .idata$6                   0000000180004796     ucrt:api-ms-win-crt-runtime-l1-1-0.dll
 0002:000017b8       .idata$6                   00000001800047b8     ucrt:api-ms-win-crt-stdio-l1-1-0.dll
 0003:00000040       ?__proc_attached@@3HA      0000000180005040     MSVCRT:dll_dllmain.obj
 0003:00000050       GS_ExceptionRecord         0000000180005050     MSVCRT:gs_report.obj
 0003:000000f0       GS_ContextRecord           00000001800050f0     MSVCRT:gs_report.obj
 0003:000005f0       ?is_initialized_as_dll@@3_NA 00000001800055f0     MSVCRT:utility.obj
 0003:000005f1       ?module_local_atexit_table_initialized@@3_NA 00000001800055f1     MSVCRT:utility.obj
 0003:000005f8       ?module_local_atexit_table@@3U_onexit_table_t@@A 00000001800055f8     MSVCRT:utility.obj
 0003:00000610       ?module_local_at_quick_exit_table@@3U_onexit_table_t@@A 0000000180005610     MSVCRT:utility.obj
